:100000000C9471220C949D220C949D220C949D22A0
:100010000C949D220C949D220C949D220C949D2264
:100020000C949D220C949D220C949D220C949D2254
:100030000C949D220C94224B0C949D220C949D2296
:100040000C949D220C949D220C949D220C949D2234
:100050000C949D220C949D220C949D220C949D2224
:100060000C949D220C949D220C949D220C949D2214
:10007000161A0102030405060708090A0B0C0D0EE7
:100080000F10110203040512131415161718191A6C
:100090001B1C1D1E1F202122231415161724252684
:1000A0002728292A2B2C2D2E2F3031323334352678
:1000B000272829363738393A3B3C3D3E3F404142BC
:1000C000434445464738393A3B48494A4B4C4D4EE4
:1000D0004F505152535455565758594A4B4C4D5AFC
:1000E000131415161718191A1B1C1D1E1F20212268
:1000F00023141516172425262728292A2B2C2D2EC4
:100100002F30313233343526272829363738393ADB
:100110003B3C3D3E3F404142434445464738393AE7
:100120003B48494A4B4C4D4E4F50515253545556F3
:100130005758594A4B4C4D5A131415161718191A7B
:100140001B1C1D1E1F2021222314151617242526D3
:100150002728292A2B2C2D2E2F30313233343526C7
:10016000272829363738393A5B5C5C5C5C5C5C5C20
:100170005C5C5C5C5C5D393A3B48494A4B4C5E00D8
:1001800000000000000000000000005F4B4C4D5AD2
:100190001314151660616161616161616161616182
:1001A00061621516172425262728292A2B2C2D2E87
:1001B0002F30313233343526272829363738393A2B
:1001C0003B3C3D3E3F404142434445464738393A37
:1001D0003B48494A4B4C4D4E4F5051525354555643
:1001E0005758594A4B4C4D5A131415161718191ACB
:1001F0001B1C1D1E1F202122231415161724252623
:100200002728292A2B2C2D2E2F3031323334352616
:10021000272829363738393A3B3C3D3E3F4041425A
:10022000434445464738393A3B48494A4B4C4D4E82
:100230004F505152535455565758594A4B4C4D5A9A
:10024000131415161718191A1B1C1D1E1F20212206
:1002500023141516172425262728292A2B2C2D2E62
:100260002F30313233343526272829363738393A7A
:100270003B3C3D3E3F404142434445464738393A86
:100280003B48494A4B4C4D4E4F5051525354555692
:100290005758594A4B4C4D5A636465666768696A9A
:1002A0006B6C6D6E6F707172736465666774160344
:1002B000755C5C5C5C5C5C5C5C5C5C5C5C5C5C5C65
:1002C0005C5C5C5C5C765E0000000000000000008E
:1002D00000000000000000000000007778797979C4
:1002E000797979797979797979797979797979797E
:1002F000797A16037B7C7D7E7F80818283848586EC
:100300008788898A8B8C8D8E8F9091929394959605
:100310009798999A9B9C9D9E9FA0A1A2A3A4A5A6F5
:10032000A7A8A9AAABACADAEAFB0B1B2B3B4B5B6E5
:10033000B7B8B9BABBBC0000000000000000000064
:1003400000000000000000000000000000000000AD
:10035000000000000000000000000000000000009D
:1003600000000000000073736B6B6B6B7320282818
:1003700028287320202020207318182820206B287C
:10038000282028186B2820182820732818182820BF
:100390007320281818186B73736B73731828201840
:1003A0002820201828281818201828202018182855
:1003B0002020201818182020181820201818181885
:1003C0002020182828286B6B7373736B181828204B
:1003D0001818182820202020282018181820282035
:1003E000181818181820201818281818202828203D
:1003F0002818282020206B6B737373731818181833
:1004000018282018182828182020182820282820E4
:1004100018181820202018282818201828202018FC
:100420001818282018286B73736B6B732020201802
:1004300018281828202018182818282020202018CC
:10044000181828281818282820202828202020209C
:10045000202018181818736B73736B6B20182820E2
:100460002828182820202020202020181828281884
:100470001828282020281828201820202828181874
:100480001820202028186B6B6B73736B2828182892
:10049000201820202018282820202018282028185C
:1004A000182820202820181820202820202018185C
:1004B00018182020182873736B6B73732820181872
:1004C000282018181828202020182820181820184C
:1004D000282018181818182020181818181820285C
:1004E000282828182820736B6B6B7373181818183A
:1004F000181820202018182818202020182818182C
:1005000028201818182820201828282020182820EB
:1005100020201818282073736B73736B1828202001
:1005200020182818182820202028281828201820CB
:1005300020181818281818182828201828282020CB
:100540001828202018186B73736B737318282018E1
:10055000282018181828202020202020201828289B
:100560002818182820202028182820202020282873
:100570001818182020206B6B6B6B6B7328282828A9
:100580001828202020202018182820202018282073
:100590002818182820182820181818182820202073
:1005A000281818182020736B73736B6B2018282081
:1005B0001818282818181828282020182820202043
:1005C0002018282020201818182018181818181873
:1005D0001828282828187373736B6B6B2820181839
:1005E000181820202020201818181820202018184B
:1005F0001818282020181828202020282820201803
:10060000282020201818737373736B731818182818
:1006100020201828281818281828202828181818E2
:1006200018202018182828181818282020182828DA
:10063000282018282020736B6B73736B20181828E0
:1006400020182020181818282820202020201818CA
:100650002828281828282020202820202020202072
:1006600018181818182073736B6B6B6B28202828C8
:100670002828202020202020201818282020182872
:10068000282028181828201828202828181828205A
:10069000202028181818736B73736B6B2018282090
:1006A0002873182820202073202020181873281859
:1006B0001828287320281828206B20202828186B39
:1006C00018202020286B6B20202828287318202031
:1006D00020207328182020207320201818286B2829
:1006E000201818186B28202018186B28202018189C
:1006F0006B181818182818182820202020182020D7
:100700001818201818182818202018282020282009
:1007100018181820282018282820282018202020E1
:1007200020201818182820282820181820202020D9
:1007300018181820202020201818182820182828D9
:1007400018282018202018282018181818282020C9
:1007500028281818282018181818282028281818A9
:100760002820202018282018181818282018282891
:100770001828201828202018282018202018282081
:100780002018182820182018282828281828202061
:100790002020282020282818282028202028282029
:1007A0001818182018182828281818282020201869
:1007B0001828201818182818182020282028281849
:1007C0002020182020281820281828202018202031
:1007D0001828201828201828202028201828202011
:1007E0002820181818182828181828202020201821
:1007F0002020202020181818182820201828181821
:100800002820181818182820182818182820182008
:1008100018282020181820202028282018182020E8
:1008200020202818182020202020181818281820E8
:1008300028281828282020201828202018181828B0
:1008400018282828181818181818181818182828D8
:1008500018182020202018282018181818282018C8
:100860002828182820182820201820201820201890
:100870002820201818282820201828282820182860
:100880002020201828202028201828202820201860
:100890002820181828201818282828201828202050
:1008A0002018182820182828281818202020202848
:1008B0002818281818202028202828182820182030
:1008C0002020182828182820182820182820182820
:1008D0001818282018182028282818182020202028
:1008E0002018182020202018201818282020201830
:1008F0001818282020201818282020201818282010
:1009000018181828202028202020202820201818F7
:10091000202018182818182018282020181818180F
:1009200018202828182828202020182020201818CF
:1009300018181828282828201818181820201818DF
:1009400028282020202020201828201818181828AF
:100950002018282818282018282018282020182097
:1009600018182820201818182820201818182820AF
:100970001828182820182820182820182820182877
:100980002018282020182820181820182820182877
:10099000182820181828282828282818202020203F
:1009A000202820282818182028202028281818183F
:1009B0001820202028282818282020202018282027
:1009C0002018181828201820202828282818202027
:1009D0002020202818202020282020181828182817
:1009E000201818181828202018181828202018183F
:1009F00018181818182828181820207320282818C4
:100A0000207318202028187328182820206B2020F5
:100A10001828206B282018282073282018282073D5
:100A200028201818186B73281828282873201828CD
:100A300020207318181818206B18282820187318ED
:100A40002020202073201820202073201818181828
:100A50006B1828282818281828282820201818203B
:100A60002018202828181828202020182820181896
:100A70001828201818282818282828202018282066
:100A80002020182820202020281828201820202066
:100A90001828281820201828201820181818181886
:100AA000182828281818182820202018181820205E
:100AB0002018282828182018182820202020182836
:100AC0002018202020181828282020181828181846
:100AD000182820181828282020181828202018281E
:100AE0001818201828202018182820181818182836
:100AF0002020202018282020202018181818281816
:100B000018282828182828202020282020201818D5
:100B100020201818282818182828182818282020D5
:100B200018281820201818181818181828282828E5
:100B300028182020202020201820181820201818DD
:100B4000281818182828282828182828202020188D
:100B500018201820202828182018202020182020AD
:100B600018181828202018282818181828202018A5
:100B7000281820201828282020202818201818207D
:100B80002020182828182020282020182018201875
:100B90001818182828281818182828202018181875
:100BA000202020182828282020181828182820203D
:100BB000182818282020201818182820201828283D
:100BC000181818282020182828202020182820202D
:100BD000281818182018202020181828201818184D
:100BE000182818282020182818282020181820181D
:100BF00028181828201818282820182828202020ED
:100C000028202020181820181818282820201828F4
:100C10002020202018202018181818181818282804
:100C200028282818202020202020181818182020D4
:100C300028282818181818282828281818282020A4
:100C400020181818182020282828201820202020B4
:100C500020201818182020201828181818182820C4
:100C6000282828182020282828202020182020186C
:100C70001820281818282818201828202018182884
:100C80002018181828182828181820182820201884
:100C9000182820202018281828202018202018285C
:100CA0002020202018282020201818182820182854
:100CB0002828181818282020182818182020182844
:100CC0002828281818181828202020181828201834
:100CD0001818201818282020201818282020182834
:100CE0002018281828202018182820201828282004
:100CF000201828202020182820181818182820200C
:100D0000182818282020182018181818181818281B
:100D100028282828282020202020202018181818CB
:100D200018182828281828281828282820201828A3
:100D300020202018181818201818282820182818DB
:100D400020202020202018202020202018181818CB
:100D50001818282828181818282818731828202048
:100D6000187318202018186B1818181828732828BA
:100D70002818207320202020187318182020186BA2
:100D80002818181828736B28202020206B18182882
:100D900020207328181828207320201828206B2062
:100DA000201818186B1818282828732818282020AD
:100DB0007320181818181820182820201818282010
:100DC000201818282020201818282020182828202B
:100DD000181828202020201828202020201828201B
:100DE000182020182820181828202018282018201B
:100DF000201828201820182820201818281820200B
:100E000018282020202018282020201828202018EA
:100E100018182820181828281818282028201828DA
:100E200020202020182020182020181818281818F2
:100E300018182820182828182820282020181818C2
:100E40002820182828282018282820201828202082
:100E500018182820201828282020181828202018A2
:100E6000282818281828202020181828202018287A
:100E7000182820181828202018282020181818189A
:100E8000182828282828181820202020201820205A
:100E90001820201828201818182820182828182862
:100EA000201828201818202018201828202018186A
:100EB000282028201828202028201828202018182A
:100EC000282018182828202020182020202020182A
:100ED000181818202018202018182820201828203A
:100EE000182020182820182018282020181828201A
:100EF00020201828282020201828282020182820E2
:100F000028201818282020182828181820182820E9
:100F100018281828202018202818202018182020E9
:100F200018181818202018282818201828202018E9
:100F300018182820182828202018282820201828A9
:100F400020202018282020181828202018182820B1
:100F50002018282828201828202018181828202091
:100F60002828182820182020202018281818181899
:100F70001818282828282828282020202020182849
:100F80002020182020182820181818282018282871
:100F90001828201828202020202018201828202059
:100FA0001818181828201828201828201828201861
:100FB0001818282018282828202018282020202029
:100FC0001818181818201828202018182820201859
:100FD0002820202020182820202018282020181819
:100FE0002820202020182820202020182820201801
:100FF0002018282018182820201828281820201801
:1010000028201820182820201818281820201828F0
:1010100020201818182820201828282020182820D8
:1010200028201818282018182820201818282020D0
:1010300018281820201828201818182820201818D8
:1010400028202018281828201828201818181828B0
:101050001828282818282828202020202020181880
:101060001818201828282828181828202020282870
:101070001828202020202018282020201828201878
:101080002018182820181828202020201818182880
:101090002020282818182820202020182820182050
:1010A0002018181818181828282828281828202048
:1010B0002820181818182020182820731818181815
:1010C000187328282828186B20202020206B202027
:1010D0001820206B28201818187320182828187337
:1010E00020182820186B7320181818187320282827
:1010F00028287320202020207318182820206B28EF
:10110000282028186B282018282073281818282031
:101110007320281818181828201828201828201894
:1011200028202018282818182018282020181828C7
:1011300020202018181820201818202018181818F7
:1011400020201828282818182820201818182820A7
:1011500018181828202020202820181818202820A7
:1011600018181818182020181828181820282820AF
:10117000281828202020181828202020181818188F
:101180001828201818282818202018282028282057
:10119000181818202020182828182018282020186F
:1011A0001818282018281828201818282020201857
:1011B000182818282020181828182820202020183F
:1011C000181828281818282820202828202020200F
:1011D000202018181818201828201818201828203F
:1011E00028281828202020202020201818282818F7
:1011F00018282820202818282018202028281818E7
:1012000018202020281818181828201828281828EE
:1012100020182020201828282020201828202818CE
:1012200018282020282018182020282020201818CE
:1012300018182020182828201818282028201818C6
:1012400028201818182820202018282018182018BE
:1012500028201818181818202018181818182028CE
:101260002828281828202018181828201818181896
:10127000181820202018182818202020182818189E
:10128000282018181828202018282820201828205E
:10129000202018182820202018282018182820205E
:1012A000201828181828202020282818282018203E
:1012B000201818182818181828282018282820203E
:1012C0001828202018181828201828201828201836
:1012D000282018181828202020202020201828280E
:1012E00028181828202020281828202020202828E6
:1012F0001818182020201818181818282828282806
:1013000018282020202020181828202020182820E5
:1013100028181828201828201818181828202020E5
:1013200028181818202020182820181820182820DD
:1013300018182828181818282820201828202020B5
:1013400020182820202018181820181818181818E5
:101350001828282828182820201818182820181895
:1013600018182020202020181818182020201818BD
:101370001818282020181828202020282820201875
:10138000282020201818282020201828181818286D
:101390002020182828181828182820282818181855
:1013A000182020181828281818182820201828284D
:1013B000282018282020201818282018201818283D
:1013C000201820201818182828202020202018183D
:1013D00028282818282820202028202020202020E5
:1013E0001818181818202820181818182820282825
:1013F00028282020202020202018182820201828E5
:1014000028202818182820182820282818182820CC
:1014100020202818181820182820186B2018282099
:1014200028731828202020732020201818732818CB
:101430001828287320281828206B20202828186BAB
:1014400018202020286B2828F6F6F6F628F6ADADF1
:10145000ADADF6AD5B5B5B5BF65B5B000000F65B26
:1014600000000000F65B00000000F65B00000000DA
:10147000F65B00000000F6F6F6F6F6F6ADADADADA3
:10148000ADAD5B5B5B5B5B5B0000000000000000E0
:10149000000000000000000000000000000000004C
:1014A000000000000000F6F6F6F62828ADADADAD60
:1014B000AD285B5B5B5BAD100000F65B5B10000072
:1014C00000F65B10000000F65B10000000F65B10F9
:1014D000000000F65B10F65B00000000F65B000009
:1014E0000000F65B00000000F65B00000000F65B09
:1014F00000000000F65B00000000F65B000000004A
:10150000F65B00000000000000F65B10000000F633
:101510005B10000000F65B10000000F65B1000009E
:1015200000F65B10000000F65B10000000F65B1098
:10153000000000F65B10F65B00000000F65B0000A8
:101540000000F65B00000000F65BAD000000F65BFB
:10155000ADF6F6F6F65B5BADADAD28AD5B5B5B5B08
:1015600028281010101000000000000000000000EB
:101570000000000000000000000000000000F6F67F
:10158000F6F6F6F6ADADADADADAD5B5B5B5B5B5B53
:10159000101010101010000000F65B10000000F694
:1015A0005B10000000F65B100000F6AD5B10F6F675
:1015B000AD5B5B10ADAD5B5B10285B5B5B10282007
:1015C0001010102820206B20202828287318202095
:1015D00020207328182020207320201818286B281A
:1015E000201818186B28202018186B28202018188D
:1015F0006B6B6B6B6B731818282020202018202031
:1016000018182018181828182020182820202820FA
:1016100018181820282018282820282018202020D2
:1016200073736B6B6B7320282820181820202020E0
:1016300018181820202020201818182820182828CA
:1016400018282018202018282018181818282020BA
:1016500073736B6B737318181818282028281818C0
:101660002820202018282018181818282018282882
:101670001828201828202018282018202018282072
:10168000736B6B73736B2018282828281828202068
:10169000202028202028281828202820202828201A
:1016A000181818201818282828181828202020185A
:1016B0006B73736B6B6B2818182020282028281850
:1016C0002020182020281820281828202018202022
:1016D0001828201828201828202028201828202002
:1016E00073736B6B6B6B2828181828202020201828
:1016F0002020202020181818182820201828181812
:1017000028201818181828201828181828201820F9
:101710006B7373736B6B20202028282018182020EF
:1017200020202818182020202020181818281820D9
:1017300028281828282020201828202018181828A1
:101740006B7373736B6B18181818181818182828EF
:1017500018182020202018282018181818282018B9
:101760002828182820182820201820201820201881
:101770007373736B6B73282020182828282018286F
:101780002020201828202028201828202820201851
:101790002820181828201818282828201828202041
:1017A000736B6B73736B282828181820202020284F
:1017B0002818281818202028202828182820182021
:1017C0002020182828182820182820182820182811
:1017D0006B6B73736B6B202828281818202020202F
:1017E0002018182020202018201818282020201821
:1017F0001818282020201818282020201818282001
:101800006B6B6B73737328202020202820201818FE
:101810002020181828181820182820201818181800
:1018200018202828182828202020182020201818C0
:101830006B6B6B73737328201818181820201818F6
:1018400028282020202020201828201818181828A0
:101850002018282818282018282018282020182088
:101860006B6B7373736B18182820201818182820B6
:101870001828182820182820182820182820182868
:101880002018282020182820181820182820182868
:101890006B73736B6B73282828282818202020204E
:1018A0002028202828181820282020282818181830
:1018B0001820202028282818282020202018282018
:1018C000736B6B6B7373182020282828281820202E
:1018D0002020202818202020282020181828182808
:1018E0002018181818282020181818282020181830
:1018F0006B6B6B6B6B7328181820207320282818CB
:10190000207318202028187328182820206B2020E6
:101910001828206B282018282073282018282073C6
:1019200073736B6B6B6BF6F6F6F6F6F6F6ADADAD64
:10193000ADADF65B5B5B5B5BF65B00000000F65BEE
:1019400000000000F65B00000000F65B00000000F5
:10195000F65B00000000F6F6F6F6F6F6ADADADADBE
:10196000ADAD5B5B5B5B5B5B00000000F65B0000AA
:101970000000F65B00000000F65B00000000F65B74
:1019800000000000F65B00000000F65B00000000B5
:10199000F65B00000000F65B00000000F65B000054
:1019A0000000F65B00000000F65B00000000F65B44
:1019B00000000000F65BF65B00000000F65B000034
:1019C0000000F65B00000000F65B00000000F65B24
:1019D000F6F6F6F6F6ADADADADAD5B5B5B5B5B5BB6
:1019E00000000000000000000000000000000000F7
:1019F0000000000000000000000000000000F6F6FB
:101A0000F6F6F6F6ADADADADADAD5B5B5B5B5B5BCE
:101A100000000000000000000000F65B0000000075
:101A2000F65B00000000F65B00000000F65BF6F6D7
:101A3000F6F6F65BADADADADAD5B5B5B5B5B5B5B8B
:101A40000000000000000949094909520909490933
:101A500049094909491249520909490949120949DB
:101A600009094949490949521252095252525252DE
:101A70000949090949094952525252525252525285
:101A8000525B1252525B52524952125252520952F6
:101A9000495252525252521252525252525252526F
:101AA0005212491249125B5B5B5B5B5B525B5B52A0
:101AB00052525B5252520000525252520000525245
:101AC0005B520000525252520000525252520000D9
:101AD0004912525200005B5B5B9B5B5B5252525B54
:101AE0009BA40000AD5B5B5B0000AD5B5B9B0000FB
:101AF000AD5B9B640000AD5B5B5B0000AD5B9B5B23
:101B00000000AD5B5B5B5B5B9B5B9B649B525252DB
:101B100052525B52000000005B52000000009B52DA
:101B2000000000005B52000000009B52000000001B
:101B30005B52000000009B64A4A4A4A452A4AD5274
:101B40005252ADA4A4520000ADA4A4520000ADA412
:101B500064520000ADA4A452ADADAD64A4A4A4A48D
:101B6000ADA4A4A4ADA4ADADADADADAD5252525235
:101B700052520000000000000000000000000000C1
:101B800000000000ADADADADAD00ADA4A4520000AD
:101B9000A4A452000000ADADADADADAD5252525255
:101BA0005252000000000000000000000000000091
:101BB000000000000000000000AD00000000ADB615
:101BC000000000ADF6F6ADADADADB6AD52B65252B9
:101BD0005252ADB652000000ADAD52000000ADB69D
:101BE00052000000F6B652000000F6B652000000A7
:101BF000B6F652000000F6B6F6B6F6B6525252529B
:101C00005252000000000000000000000000000030
:101C10000000000000ADADADADAD00ADF6FFF6FFCC
:101C200000AD52525252F6F6FFF6FFFF5252525298
:101C300052520000000000AD0000000000AD0000A6
:101C4000000000ADADADADADADADFFFFFFFFFFFFDF
:101C50005252ADF6FFFFFFFFFFFFFFFFFF52525250
:101C60005252FF5200000000FF5200000000FF52DD
:101C700000000000F65200000000FF5200000000CB
:101C8000F65200000000FFF6F6F6B6F65252525237
:101C900052520000000000000000000000000000A0
:101CA00000000000ADADADADAD52ADF6B6F6B6522A
:101CB000AD5252525252B6F6ADADADAD5252525235
:101CC00052F600000000ADB600000000ADAD00000F
:101CD0000000ADB600000000ADB600000000ADF69B
:101CE00000000000ADB6ADADADADADADAD525252E0
:101CF0005252AD5200000000AD5200000000ED5203
:101D000000000000B65200000000ED52000000008C
:101D1000AD5200000000ADADADA4ADA45252525280
:101D2000525200000000000000000000000000000F
:101D300000000000ADADADADAD52ADADADADAD523D
:101D4000ADADADA4A452A4A4A4A4A4A452525252D2
:101D5000525B00000000ADA400000000ADA4000034
:101D60000000AD5B00000000ADA400000000ADA4C9
:101D700000000000AD64A464A45BA45B5252525204
:101D8000529B5200000000AD5200000000005200C3
:101D900000000000A452000000005BA452000000FC
:101DA000A45BA45200005B5B5B5B5B5B5B9B5B9B30
:101DB0005B525B5B5B5B5200AD9B5B52000000AD16
:101DC00052000000000000000000000000000000C1
:101DD000000000000000525B525B525252525252BD
:101DE0005B5B000000AD0000000000AD5B00000088
:101DF00000AD52000000AD5B5B0000AD9B5B5B5B28
:101E0000AD5B5B5B525B525252525252525B52522A
:101E100052520052005252525B52000052005B522A
:101E2000005200525B5B0052525252525B5252526D
:101E3000525B525252525252524952095209521254
:101E400049520052525252090009490909490052A7
:101E50000949090900525252494952124909520985
:101E600012495209490909090949094949524912BE
:101E7000525252095252495209524952521249126F
:101E80004912495252495252124952125252525216
:101E900009490949095209495249525252124912F3
:101EA000525252525252125252525252525249129B
:101EB000525252525252095212525252525252528B
:101EC00012525252525252525252000052525B52CD
:101ED00000005252525200005252525200005252CE
:101EE0005B520000525252520000525B52520000AC
:101EF0005B525B5200000000AD5B5B9B0000AD5B82
:101F00005B5B0000AD5B9B5B0000AD5B5B5B00005F
:101F1000AD5252520000000000000000000000001E
:101F20000000000000005B52000000009B52000017
:101F300000005B52000000009B5200000000525263
:101F40000000000000000000000000000000000091
:101F5000000000000000ADA4A464A4ADADA464A47E
:101F600064A4AD64A4A4A452ADA4A4A45200ADA4DE
:101F700064520000ADA4A4520000AD64A45200005D
:101F8000ADA4A4520000A4520000000052000000C2
:101F900000000000000000000000000000AD000094
:101FA0000000AD5200000000000000000000000032
:101FB0000000000000000000ADF6B6F600ADF6ED42
:101FC000B6B6ADB6B6B6F6F6EDB6F6ADF6B6525254
:101FD00052525252000000000000000000000000B9
:101FE000000000000000F6F652000000B6F65200B5
:101FF0000000F6B652000000B6F65200000052B6DD
:1020000052000000ADF652000000ADB652000000D4
:10201000ADB652000000000000000000000000000B
:10202000000000ADADADADAD00ADF6B6F6B600AD9D
:102030005252525200000000000000000000000058
:102040000000000000000000ADFFFFF60000ADFF43
:10205000FFFFADADADF6FFF6F6B6F6B6FFF652529F
:10206000525252520000000000AD0000000000ADCE
:102070000000000000ADFF5200000000FF52000011
:102080000000FF5200000000BF5200000000F652A6
:1020900000000000FF5200000000F65200000000A7
:1020A000FF520000000000000000000000000000DF
:1020B0000000ADADADADAD52ADF6FFF6F652AD528E
:1020C00052525252000000000000000000000000C8
:1020D00000000000000000000000ADAD000000ADF9
:1020E00052AD00000000ADF600000000ADB60000EB
:1020F0000000ADAD00000000ADED00000000ADB689
:1021000000000000ADF6AD5200000000ED520000EE
:102110000000B65200000000ED5200000000B65270
:1021200000000000AD5200000000F6520000000068
:10213000B65200000000ADADA4A46452ADADADA494
:10214000A452ADADADADAD52ADADA4A4AD52AD5246
:102150005252525200000000000000000000000037
:1021600000000000000000000000ADA4000000001E
:10217000ADA400000000ADA400000000ADA400006C
:102180000000ADA400000000AD6400000000ADA49C
:1021900000000000ADA4A4A4A464520064A4649B45
:1021A0005200A45BA49B520064A49B5200009B6459
:1021B00052000000A4520000000052000000000085
:1021C0005200000000AD0000000000AD0000000063
:1021D00000AD0000000000AD0000000000000000A5
:1021E0000000000000ADAD000000ADA4A45200004E
:1021F000A45B5B5B52005B52525252525B5B5B5280
:102200005B525B5B5B5B5B5BAD5B5B5B525200ADF0
:102210005B9B5B5B0000AD5B5B52000000AD5B5BFA
:10222000000000AD5B525252525212495252525269
:1022300052125B52525252525252525252525252B5
:10224000525212525B5252525252525B525252529C
:10225000525252521252495209520952524952494B
:10226000490912521252095249524949094952091F
:1022700052124909525249525252124912520949B4
:102280004912494909524909490952090949094963
:10229000095209094909524949525252525252525D
:1022A000525252520909521252524952495249123B
:1022B000094912491252495212525252524952522B
:1022C000525212525252525252525252525B5B521C
:1022D00052525252525252525252525252525252DE
:1022E00052125252525252525252ADAD5252525258
:1022F0005B5B5B5B5B5B5B9B52525B52525B525224
:102300005252525252525252525252525252525BA4
:102310005B525B5B5B52ADADADADADAD5B5B5B5B33
:102320005B5B5B9B5B9B5B005B5B5BA45B005B5BEA
:102330009B5B5B005252525B5B00525B5B525B00EB
:102340005B5B525B5B5BADADADADADAD5B5BA464A8
:10235000A4A40000005B000064A400A400645B9BD4
:10236000006400005B5B00A400640000005B00A44C
:102370005B9B64A464A4ADA4A452ADADA4A4A4AD1D
:10238000ADAD0000A4000000A400A400A4AD0000B6
:10239000A4000000A4A4A400A4ADA4A4AD00000067
:1023A00064A464A4A4A4ADADADADADADADADADAD13
:1023B000ADAD00AD00ADAD00ADAD0000ED00A4AD24
:1023C00000AD0000ADAD00ADAD0000A400ADAD00AE
:1023D000A4A4A4A4A4ADADADADADADADADADB6ED11
:1023E000ADF6ADADAD000000F6ADF600F6ADADADAD
:1023F000AD000000ADADADEDADB6ADEDB600000089
:10240000ADADADB6EDB6ADAD52ADADADB6F6F6F621
:10241000F6F600B600000000F6ED00B6B60000B615
:1024200000ADF60000AD00F6B60000F600000000BA
:10243000F6B6F6F6F6F6ADADADADADADF6F6FFF629
:10244000FFFFF600B6FF00F6F600F6F600F6F6001F
:10245000FFB600FFB600F6FF00BFF600000000F672
:10246000F6F6F6F6B6F6ADADADADADADFFFFFFFFDE
:10247000F6FF00000000F60000F6FF00F600000086
:1024800000FFFF0000F6FF00FF0000FFF600F6006F
:10249000B6F6BFF6BFFFFF52ADADADADF6FFFFFF25
:1024A000FFFF000000FF0000F6FFFFF600F6FFFF51
:1024B000F6FF0000F6FFFFFF00F6000000FF00003F
:1024C000B6F6FFB6FFFFADADADADADADFFFFFFF6AC
:1024D000FFF60000B6F6B600F6FFF6FFF60000B60F
:1024E000F6B6B600FFFFF6F6F6000000F6BFF600FF
:1024F000F6B6FFFFF6FFADADADADADF6F6F6F6F60E
:10250000B6B6000000B60000F6F6B6F600B6B6B6EF
:10251000ADAD00EDF6F6B6F600B6000000B6000070
:10252000F6FFB6F6F6B6F652ADADADADB6F6ADAD5C
:10253000ADAD0000F600ADEDB600AD0000ADAD00F4
:10254000AD00AD00ED00AD00ADAD0000AD00ADEDF6
:10255000F6ADB6EDADADADADADADADADADADADAD19
:10256000A4AD00AD0000000000AD00ADA4AD00AD15
:102570000000000000ADADADA40000AD0000000003
:10258000ADADADADADADADADADADADA4A4ADA4A49F
:1025900064A4AD0000000064A400A4A400A4A400EE
:1025A00064A40064A400A46400A4AD00000000A41E
:1025B000A4ADADADADA452ADADADAD5BA464A464AE
:1025C000A4A400A45BA45B00005BA45B5B0000A46C
:1025D0005BA45B0000A45B5B9B00000000005B0051
:1025E000A4A4A464A4A45B5B9B5B5B52A4A45B9BBC
:1025F0005B5B0000009B5B5B5B5B9B5B5B5B000072
:102600005B5B5B5B5B5B5B5B9B520000005B5B5BF4
:10261000649B5B5B9B5BADADADAD52525B5B5B5B4B
:102620005B5B5B5B5B5252529B5B525B5B525B5BE7
:102630005B52525B52525B5B52525B5B525B5B5B29
:102640005B5B5B5B5252525252124952525252528F
:10265000525252525252525252525252125252529A
:10266000525252525B525B52525252525252525238
:1026700052525252521209490912490952525249B0
:102680001249525209524909094909490949525204
:1026900052520949525212495209124952094909E2
:1026A0004949090949090000000000000000000034
:1026B000000000000000000000000000000000001A
:1026C000000000000000000000000000000000000A
:1026D0000000000000000000FF00000000FFFFFFFE
:1026E000000000FFFFFF00000000FF0000000000EE
:1026F000FF0000000000000000000000FF000000DC
:10270000000000000000FFFF00FFFF00FFFF00FFD0
:10271000FF00FF0000FF00000000000000000000BC
:1027200000000000000000000000000000000000A9
:1027300000000000000000000000000000FF00FF9B
:102740000000FFFFFFFFFF0000FF00FF000000FF91
:1027500000FF0000FFFFFFFFFF0000FF00FF000081
:1027600000000000000000FF0000000000FFFFFF6D
:102770000000FF000000000000FFFF00000000005C
:1027800000FF0000FFFFFF0000000000FF0000004E
:10279000000000000000FFFF0000FF00FFFF00003E
:1027A000FF00000000FF00000000FF00000000FF2D
:1027B00000000000FF0000FFFF00FF0000FFFF001F
:1027C00000000000000000FF00000000FF00FF000C
:1027D0000000FF00FF00000000FF00000000FF00FD
:1027E000FF00FF00FF0000FF000000FFFF00FF00F0
:1027F00000000000000000FFFF00000000FFFF00DD
:10280000000000FF000000000000000000000000C9
:1028100000000000000000000000000000000000B8
:102820000000000000000000FF00000000FF0000AA
:10283000000000FF0000000000FF0000000000FF9B
:102840000000000000FF000000000000FF0000008A
:1028500000000000000000FF000000000000FF007A
:1028600000000000FF0000000000FF00000000006A
:10287000FF0000000000FF00000000FF000000005B
:1028800000000000000000000000000000FF00FF4A
:10289000000000FFFFFF0000FFFFFFFFFF0000FF41
:1028A000FFFF000000FF00FF00000000000000002C
:1028B0000000000000000000000000000000FF0019
:1028C00000000000FF000000FFFFFFFFFF0000000E
:1028D000FF0000000000FF000000000000000000FA
:1028E00000000000000000000000000000000000E8
:1028F00000000000000000000000000000000000D8
:102900000000000000FFFF00000000FFFF000000CB
:1029100000FF0000000000000000000000000000B8
:102920000000000000000000FFFFFFFFFF000000AC
:102930000000000000000000000000000000000097
:102940000000000000000000000000000000000087
:102950000000000000000000000000000000000077
:102960000000000000FFFF00000000FFFF0000006B
:102970000000000000000000000000000000000057
:10298000FF00000000FF00000000FF00000000FF4B
:1029900000000000FF000000000000000000000038
:1029A000000000000000002F2F2F00002F0000006B
:1029B0002F002F00002F2F002F002F002F002F2F70
:1029C00000002F002F0000002F00002F2F2F0000ED
:1029D00000000000000000002F000000002F2F006A
:1029E000000000002F00000000002F000000000089
:1029F0002F00000000002F000000002F2F2F0000EC
:102A0000000000000000002F2F2F00002F0000000A
:102A10002F00000000002F0000002F2F0000002FCB
:102A2000000000002F00000000002F2F2F2F2F008C
:102A3000000000000000002F2F2F00002F000000DA
:102A40002F00000000002F00002F2F2F000000009B
:102A500000002F002F0000002F00002F2F2F00005C
:102A60000000000000000000002F000000002F2FD9
:102A70000000002F002F00002F00002F00002F2F3C
:102A80002F2F2F000000002F00000000002F00005B
:102A90000000000000002F2F2F2F2F002F0000001C
:102AA00000002F00000000002F2F2F2F000000003B
:102AB00000002F002F0000002F00002F2F2F0000FC
:102AC00000000000000000002F2F0000002F000079
:102AD00000002F00000000002F2F2F2F00002F00DC
:102AE00000002F002F0000002F00002F2F2F0000CC
:102AF0000000000000002F2F2F2F2F0000000000EB
:102B00002F000000002F000000002F000000002F09
:102B100000000000002F00000000002F0000000057
:102B2000000000000000002F2F2F00002F000000E9
:102B30002F002F0000002F00002F2F2F00002F004C
:102B400000002F002F0000002F00002F2F2F00006B
:102B5000000000000000002F2F2F00002F000000B9
:102B60002F002F0000002F00002F2F2F2F0000001C
:102B700000002F000000002F0000002F2F00000099
:102B80000000000000000000000000000000000045
:102B9000000000FFFF00000000FFFF000000000039
:102BA0000000000000FFFF00000000FFFF00000029
:102BB0000000000000000000000000000000000015
:102BC000000000FFFF00000000FFFF000000000009
:102BD0000000000000FFFF00000000FFFF000000F9
:102BE00000FF0000000000000000FF00000000FFE8
:102BF00000000000FF00000000FF000000000000D7
:102C0000FF000000000000FF000000000000FF00C7
:102C100000000000000000000000000000000000B4
:102C20000000FFFFFFFFFF000000000000000000A9
:102C300000000000FFFFFFFFFF0000000000000099
:102C400000000000000000FF000000000000FF0086
:102C50000000000000FF000000000000FF00000076
:102C600000FF00000000FF00000000FF0000000067
:102C700000000000000000FFFFFF0000FF00000058
:102C8000FF0000000000FF000000FFFF0000000048
:102C9000FF0000000000000000000000FF00000036
:102CA00000000000000000FFFFFF0000FF00000028
:102CB000FF00FF00FFFFFF00FF00FF00FF00FF001D
:102CC000FFFFFF00FF000000000000FFFFFF00000B
:102CD00000000000000000FFFFFF0000FF000000F8
:102CE000FF00FF000000FF00FF000000FF00FFFFEB
:102CF000FFFFFF00FF000000FF00FF000000FF00DB
:102D0000000000000000FFFFFFFF0000FF000000C8
:102D1000FF00FF000000FF00FFFFFFFF0000FF00BB
:102D20000000FF00FF000000FF00FFFFFFFF0000AA
:102D300000000000000000FFFFFF0000FF00000097
:102D4000FF00FF0000000000FF0000000000FF0087
:102D500000000000FF000000FF0000FFFFFF000078
:102D6000000000000000FFFFFFFF0000FF00000068
:102D7000FF00FF000000FF00FF000000FF00FF0059
:102D80000000FF00FF000000FF00FFFFFFFF00004A
:102D9000000000000000FFFFFFFFFF00FF00000039
:102DA0000000FF0000000000FFFFFFFF0000FF0029
:102DB00000000000FF0000000000FFFFFFFFFF0019
:102DC000000000000000FFFFFFFFFF00FF00000009
:102DD0000000FF0000000000FFFFFFFF0000FF00F9
:102DE00000000000FF0000000000FF0000000000E5
:102DF00000000000000000FFFFFF0000FF000000D7
:102E0000FF00FF0000000000FF00FFFFFF00FF00C9
:102E10000000FF00FF000000FF0000FFFFFFFF00B9
:102E2000000000000000FF000000FF00FF000000A5
:102E3000FF00FF000000FF00FFFFFFFFFF00FF009B
:102E40000000FF00FF000000FF00FF000000FF0087
:102E500000000000000000FFFFFF00000000FF0076
:102E600000000000FF0000000000FF000000000064
:102E7000FF0000000000FF00000000FFFFFF000057
:102E800000000000000000000000FF000000000043
:102E9000FF0000000000FF0000000000FF00FF0036
:102EA0000000FF00FF000000FF0000FFFFFF000028
:102EB000000000000000FF000000FF00FF0000FF16
:102EC0000000FF00FF000000FFFF00000000FF0007
:102ED000FF000000FF0000FF0000FF000000FF00F7
:102EE000000000000000FF0000000000FF000000E4
:102EF0000000FF0000000000FF0000000000FF00D5
:102F000000000000FF0000000000FFFFFFFFFF00C7
:102F1000000000000000FF000000FF00FFFF00FFB6
:102F2000FF00FF00FF00FF00FF000000FF00FF00A8
:102F30000000FF00FF000000FF00FF000000FF0096
:102F4000000000000000FF000000FF00FFFF000085
:102F5000FF00FF00FF00FF00FF0000FFFF00FF0079
:102F60000000FF00FF000000FF00FF000000FF0066
:102F700000000000000000FFFFFF0000FF00000055
:102F8000FF00FF000000FF00FF000000FF00FF0047
:102F90000000FF00FF000000FF0000FFFFFF000037
:102FA000000000000000FFFFFFFF0000FF00000026
:102FB000FF00FF000000FF00FFFFFFFF0000FF0019
:102FC00000000000FF0000000000FF000000000003
:102FD00000000000000000FFFFFF0000FF000000F5
:102FE000FF00FF000000FF00FF000000FF00FF00E7
:102FF000FF00FF00FF0000FF000000FFFF00FF00D8
:10300000000000000000FFFFFFFF0000FF000000C5
:10301000FF00FF000000FF00FFFFFFFF0000FF00B8
:1030200000FF0000FF000000FF00FF000000FF00A5
:1030300000000000000000FFFFFF0000FF00000094
:10304000FF00FF000000000000FFFFFF0000000085
:103050000000FF00FF000000FF0000FFFFFF000076
:10306000000000000000FFFFFFFFFF000000FF0066
:1030700000000000FF0000000000FF000000000052
:10308000FF0000000000FF0000000000FF00000043
:10309000000000000000FF000000FF00FF00000033
:1030A000FF00FF000000FF00FF000000FF00FF0026
:1030B0000000FF00FF000000FF0000FFFFFF000016
:1030C000000000000000FF000000FF00FF00000003
:1030D000FF00FF000000FF00FF000000FF00FF00F6
:1030E0000000FF0000FF00FF00000000FF000000E4
:1030F000000000000000FF000000FF00FF000000D3
:10310000FF00FF00FF00FF00FF00FF00FF00FF00C7
:10311000FF00FF00FF00FF00FF0000FF00FF0000B6
:10312000000000000000FF000000FF00FF000000A2
:10313000FF0000FF00FF00000000FF00000000FF94
:1031400000FF0000FF000000FF00FF000000FF0084
:10315000000000000000FF000000FF00FF00000072
:10316000FF00FF000000FF0000FF00FF0000000064
:10317000FF0000000000FF0000000000FF00000052
:10318000000000000000FFFFFFFF0000000000FF44
:1031900000000000FF00000000FF00000000FF0032
:1031A00000000000FF0000000000FFFFFFFF000024
:1031B0000000000000000000FFFF000000FF000012
:1031C000000000FF00000000FFFF0000000000FF03
:1031D0000000000000FF000000000000FFFF0000F2
:1031E0000000000000000000FFFF000000FF0000E2
:1031F000FF00FF00FFFF00FFFF00FF0000FFFF00D8
:10320000FFFF00FF00FF0000FF000000FFFF0000C5
:1032100000000000000000FFFF000000000000FFB1
:103220000000000000FF0000000000FFFF000000A1
:1032300000FF0000000000FF000000FFFF00000092
:10324000000000000000FEFEFEFEFEFEFEFEFEFE92
:10325000FEFEFEFEFEFEFEFEFEFEFEFEFEFEFEFE8E
:10326000FEFEFEFEFEFEFEFEFEFEFEFEFEFEFEFE7E
:10327000FEFEFEFEFEFE5EAFAFAFAFB7A6151616A2
:103280001616A61516161616A61516161616A61531
:1032900016161616A61516161616A61516161616B0
:1032A000A615161616165C0CAFAFAF560B651E169C
:1032B00015090B651E1615090B651E1615090B5C05
:1032C0000A1615090B0B010001550BA5B7AFAE4946
:1032D0000B651E161509A61516161616A615161632
:1032E0001616000B1616160CB7530016160CA6660B
:1032F000AE000049A61516AFAF52A6151616154A10
:1033000014000000005E0B651E1615090B651E16E5
:103310001509535F15161509535F1516150967151D
:1033200016161509661516161509671516160908D5
:103330005C0000000155AFAFAFAFAFAF151616166A
:10334000150A15161616150A0000000000001516BD
:103350000A15161615160A15161615160A15161636
:10336000000000000000AFAFAFAFAFAE16161616EC
:103370001509161616161509000000000008161586
:103380000A16165516150A16165516150A16165546
:1033900000000000000815161616150A1516161658
:1033A000150A15161616150A00000000000015165D
:1033B0000A15161615160A15161615160A151616D6
:1033C000000000000000161616161509161616162F
:1033D0001509161616161509000000000008161526
:1033E0000A16165516150A16165516150A161655E6
:1033F000000000000008FEFE0000FEFEFE005F046C
:1034000000FE005FFF070400000707070400000636
:1034100007060400000406060400FE00040400FE83
:10342000FEFE0000FEFEFEFE0000FEFEFE00EA992B
:1034300000FE00EAFFE2490000E2E2E249000099F2
:10344000E2994900004999994900FE00494900FE66
:10345000FEFE0000FEFEFEFE0000FEFEFE007D21E0
:1034600000FE007DFF3119000031313119000021CB
:1034700031211900001921211900FE00191900FE3F
:10348000FEFE0000FEFEFEFE0000FEFEFE00F786D1
:1034900000FE00F7FFC74C0000C7C7C74C000086FE
:1034A000C7864C00004C86864C00FE004C4C00FE4B
:1034B000FEFE0000FEFEE3E3E3E3E3E3E3E3E3E336
:1034C000E3E3E3E3E3E3E3E3E3E3E3E3E3E3E3E3CC
:1034D000E3E3E3E3E3E3E3E3E3E3E3E3E3E3E3E3BC
:1034E000E3E3E3E3E3E3000000000000000000008A
:1034F00000000000000000000000000000000000CC
:1035000000000000000000000000000000000000BB
:10351000000000000000FEFFADFEFEFEFFFFFFAD5D
:10352000FEFEFFFFFFA400FEADFFADA40000A4ADB2
:10353000A4A40000FEA4A4000000FEFE0000000001
:10354000FEFEFE0000FE0000000000000000000083
:10355000000000000026262600000027FF270000AC
:10356000FF0D0D0B0000000B0B0B0000000B0B0BF5
:10357000000000000000000000000000000000004B
:10358000000052A4A4A4A4A452FFFFFFFFFF52A472
:10359000A4A4A4A400525252525200525252525267
:1035A000000000000000000000000000000000001B
:1035B00000005226262600005227FF270000520D49
:1035C0000D0BFF00000B0B0B0000000B0B0B0000A2
:1035D000000000000000A4A4A4A4A4A4A4A4A4A483
:1035E000A4A4A4A4A4A4A4A4A4A4A4A4A4A4A4A49B
:1035F000A4A4A4A4A4A4A4A4A4A4A45B5B5B5B5BF8
:10360000000000000000A4A4A4A45200A4A4A4A448
:103610005200A4A4A4A45200A4A4A4A45200A4A44C
:10362000A4A45200A4A4A4A452005B5B5B5B520060
:103630000000000000001D1D1D1D1D1D1D1D1D1D68
:103640001D1D1D1D1D1D1D1D1D1D1D1D1D1D1D1DAA
:103650001D1D1D1D1D1D1D1D1D1D1D1515151515C2
:103660000000000000001D1D1D1D0D001D1D1D1D65
:103670000D001D1D1D1D0D001D1D1D1D0D001D1D01
:103680001D1D0D001D1D1D1D0D00151515150D0011
:10369000000000000000A8A8A8A8A8A8A8A8A8A89A
:1036A000A8A8A8A8A8A8A8A8A8A8A8A8A8A8A8A89A
:1036B000A8A8A8A8A8A8A8A8A8A8A8A0A0A0A0A0B2
:1036C000000000000000A8A8A8A85800A8A8A8A862
:1036D0005800A8A8A8A85800A8A8A8A85800A8A852
:1036E000A8A85800A8A8A8A85800A0A0A0A0580062
:1036F000000000000000282828282828282828283A
:103700002828282828282828282828282828282839
:103710002828282828282828282828202020202051
:103720000000000000002828282818002828282841
:1037300018002828282818002828282818002828B1
:1037400028281800282828281800202020201800C1
:103750000000000000000505050505050505050537
:103760000505050505050505050505050505050509
:1037700005050505050505050505050404040404FE
:10378000000000000000050505050300050505050E
:1037900003000505050503000505050503000505EE
:1037A00005050300050505050300040404040300E2
:1037B0000000000000009898989898989898989819
:1037C0009898989898989898989898989898989879
:1037D0009898989898989898989898909090909091
:1037E00000000000000098989898500098989898C9
:1037F00050009898989850009898989850009898E9
:1038000098985000989898985000909090905000F8
:1038100000000000000095959595959595959595D6
:103820009595959595959595959595959595959548
:1038300095959595959595959595958C8C8C8C8C65
:10384000000000000000959595955300959595957D
:10385000530095959595530095959595530095959D
:10386000959553009595959553008C8C8C8C5300B1
:103870000000000000002D2D2D2D2D2D2D2D2D2D86
:103880002D2D2D2D2D2D2D2D2D2D2D2D2D2D2D2D68
:103890002D2D2D2D2D2D2D2D2D2D2D242424242485
:1038A0000000000000002D2D2D2D1B002D2D2D2D95
:1038B0001B002D2D2D2D1B002D2D2D2D1B002D2DF5
:1038C0002D2D1B002D2D2D2D1B00242424241B0009
:1038D000000000000000FFFFFFFFFF52FFADADAD95
:1038E000AD00FFADFFFFAD00FFADFFADAD00FFAD23
:1038F000FFADAD00FFADFFADAD00FFADADADAD00B7
:10390000520000000000FFA4A4A4A4A4FFFFA4A4EC
:10391000A4A4FFFFFFA4A4A4FFFFFFFFFFFFFFFF7E
:10392000FF5B5B5BFFFF5B5B5B5BFF5B5B5B5B5B57
:10393000000000000000A4A4A4A45200A4A4A45267
:103940005200A4A452525200FF52525252005B5BEA
:10395000525252005B5B5B5252005B5B5B5B5200FE
:10396000000000000000FEFE2626260DFE27272769
:10397000270D0B27FFFFFF0DFF262727270D0B26FF
:103980002626260D0B0D0D0D0D0BFE0B0B0B0B0B39
:10399000FEFE0B0B0B0BFE5B5B5B5B5B52A4A4A4FC
:1039A000A4A452FFFFFFFFFF52A4A4A4A4A400A458
:1039B000A4A4A4A4005B5B5B5B5B005B5B5B5B5BE9
:1039C0000000000000005B5B5B5B5BFEA4A4A4A4A2
:1039D000A452FFFFFFFFFF52A4A4A4A4A452A4A4D6
:1039E000A4A4A4005B5B5B5B5B005B5B5B5B5B005D
:1039F00000000000000026262626FEFE2727272797
:103A00000DFEFFFFFF270D0B272727270DFF26267B
:103A100026260D0B0D0D0D0D0B0B0B0B0B0B0B00C1
:103A20000B0B0B0B0000FEFE00000000FEFEFE0074
:103A30000000FEFEFEFE0000FEFEFEFEFEFEFEFE9E
:103A4000FEFEFEFEFEFEFEFEFEFEFEFEFEFEFEFE96
:103A5000FEFEFEFEFEFE0000000000000000000072
:103A600000000000FE000000FEFEFEFEFEFEFEFE68
:103A7000FEFEFEFEFEFEFEFEFEFEFEFEFEFEFEFE66
:103A8000FEFEFEFEFEFE0000000000000000000042
:103A90000000000000000000FEFEFEFEFEFEFEFE36
:103AA000FEFEFEFEFEFEFEFEFEFEFEFEFEFEFEFE36
:103AB000FEFEFEFEFEFE0000000000000000000012
:103AC00000FE00FE0000FEFEFEFEFEFEFEFEFEFE0E
:103AD000FEFEFEFEFEFEFEFEFEFEFEFEFEFEFEFE06
:103AE000FEFEFEFEFEFEFEFFFFFEFEFEFFFDFDFFF4
:103AF000FEFEFFFDFAFF00FEFFFAAAFF0000FFAA8C
:103B0000AAFF0000FEFFFF000000FEFE0000000014
:103B1000FEFEFE0000FEFEFFFFFEFEFEFFADA45215
:103B2000FEFEFFADA45200FEFFA45B520000AD5BA1
:103B30005B520000FE5B52000000FEFE0000000031
:103B4000FEFEFE0000FE53505249544520454E47AC
:103B5000494E452044454D4F005C323030382055A9
:103B60005A45202D2047504C20563300202020203D
:103B70005354415254203D204F5645524C41590018
:103B800053434F52455320474F45532048455245D4
:103B900021203A2900583A00593A0000000000005C
:103BA0000000000000000000000000000000000015
:103BB0000000000000000000000000000000000005
:103BC00000000000000000000000000000000000F5
:103BD00000000000000000000000000000000000E5
:103BE000000000000000000000000000000049008C
:103BF0000000495252000052525C2D0000000000AB
:103C00000000000000000000000000004000000074
:103C1000494A52004952525B1C52531C25241B2412
:103C200025251B0A0A2D1C12120A0A00000000009A
:103C3000000000404949494949525B5B5B525B1CAB
:103C40001C1312241C1209090912090909090A0A7C
:103C50000A0A0A0A13120A0A12130A0000000000D4
:103C60000092525252525213121309001C0A12129D
:103C7000401B65090A0009241B120000251C1C01B9
:103C80000025241C1C0024252424240000000000FE
:103C9000005249494000001B1352494900641C1C52
:103CA0005B4A481C651C2552491C1C652464491C40
:103CB0001C652564491C1C6D2E5C49000000000039
:103CC0000000000000004900000000535200000006
:103CD00053522500004A52252500005B25130000A1
:103CE0005B53000A1C095B1C657F374052522E2E25
:103CF0001C525C2E251B1324251C1C12002525128A
:103D00000000121B0000132E37001B37372E2E37F2
:103D1000372E2E2E2E2E2E6E6E6E1C1313120009B1
:103D2000131200001213130012251C13132E371C3C
:103D3000131313361C131B1B1B25131C1C1B1B1BD3
:103D40001C1C1C1C1C1C1C1C1C1C131312121313EB
:103D5000001313131C000913131C010037131C1349
:103D6000002E2E1C1C001C772E2500137F251C0105
:103D70000A37241C1C0A2E25250900132E2425256C
:103D8000252E252525252525252D2E251B2E2E25C1
:103D90001C1325251C1C1C1C011C1C1300011C0AC7
:103DA000000165775C016E7F6E521B25256D1C52EC
:103DB0004925251C1353001C1C1C524A001B135B75
:103DC0005B000009525C0000005B5C000000001B0F
:103DD0000000000000000000000000135B7F776E11
:103DE0006E136577766E6E1B65777676761B5BBF96
:103DF00076B67609136DBFB7B6001B125C76BF00AE
:103E000000121B125B00000000090A6E6E6E772420
:103E10001C6E6E77251C1C6E776E1C1C1C76761C27
:103E20001C2425B765646D6D1B766D6D5B09125B97
:103E30005C5B125B641213131B12121C1C1C1C1CF7
:103E4000241C1C242525242425251B0000251300C3
:103E50000064BF00096EBFBF6D6EBF6D5B12135B68
:103E600012131209000901000000002E1C090009AC
:103E70006E010009767F7F12777F7F6412BF775BC8
:103E8000121B095B121B0900001B09000000000047
:103E900000000000000000000000007F7F531313AB
:103EA0000064121B0100001B120000000000000053
:103EB0000000000000000000000000000000000002
:103EC00000000000000000000000000000000000F2
:103ED000002600000026002F0000002F0037000001
:103EE000003700FF000000FF00BF000000BF0037E8
:103EF000000037000000262600000000000000003F
:103F000000262626262600000000002F00000000C4
:103F10003700000000FF00000000BF000000003775
:103F200000000000002626262626000000000000D3
:103F3000002626262626002F00000000003700005D
:103F4000000000FFFFFFFF0000BF0000000000377F
:103F500000000000002626262626000000000000A3
:103F6000002626262600002F0000002F0037000024
:103F7000003700FFFFFFFF0000BF000000BF003759
:103F80000000003700262626260000000000000062
:103F900000000026262600002F00002F003700001A
:103FA000003700FF000000FF00BF000000BF003727
:103FB0000000370000262626000000000000000058
:103FC000002600000026002F0000002F0000370010
:103FD0003700000000FF00000000BF00BF000037F6
:103FE000000000370026000000260000000000004E
:103FF00000000000000000000000000000000000C1
:1040000000000000000000000000000000009B0015
:104010000000529BA400005B9B6D77000000000035
:104020000000000000000000000000005B00000035
:10403000E4F6FF099BEDF6FFBFA4ADBFBFBFBF769F
:104040007F7FB7B7BF7F766EB7B7BF0000000000B5
:104050000000005BB6F6F6F6FFFFFFFFBFFFFFFFB5
:10406000BFBFAEFFFFFFB7AD65FFFFB7B6AD65FFE2
:10407000FFBFB7AE6EFFFFBFB7B76500000000001F
:1040800000F6F6EDEDADA4B66D6D5C526E6565653E
:104090005265765C5C52536E246552526E25255BE8
:1040A00052772D2525526E6E2D252500000000002B
:1040B00000A49B9B4900006564A49B92006D25258C
:1040C000649349656E652E9B5224256D25655225A6
:1040D000246D2D655225256E2E64520000000000CF
:1040E0000000000000004A000000005B9B00000090
:1040F0005B5B2D0000525B2E2E00015B2D1C01002E
:104100005C5B014A654A5B1C6E7F77495B9B7777F6
:104110006D5B65776E65656D2D25255C522E2513CB
:104120000949641C09095C7F7F091C7F7F777F77C1
:104130007F77777F7F7776777F7F6E656E6EA4B6A9
:10414000FF655BA4B7BFFF526DBFBFBFFF7FBFBF9F
:10415000BFBFFFBFBFB7BFFFFF7FB7BFBFFFFF6ED0
:10416000B7BFBFFFFF77BFBFBFFFFFFFFFBFBFB737
:104170005BFFFFBFBFA464FFFFBFADA47FFFFFBF16
:10418000A4BF7FFFBFADBFBFBFFFB6BFBFBF77F745
:10419000BFBFBF7777FFBFBFBF64526D7F6E2E2D4D
:1041A0002D7F766E6E6E2E777777762E1C7F776EEC
:1041B000251C25776525251C096E6E1C0949255B84
:1041C000494A6E7F645377BF775B5C256E6E255BD3
:1041D0004A25651C1B5B002524245B53001C1B5BCC
:1041E0005C00000A5B640000006464000000005C86
:1041F00000000000000000000000005B5C7FBF7753
:10420000765C6D7FB777775C6D7FBF77775C64BFD7
:10421000BFBFBF0A5C6EBFBFBF0065646DBFBF009C
:10422000005B6D646D00000000125B7777777F6E36
:104230006E77777F766D7677BF776D6E76BF7F6DA1
:104240006E767FBF7676BFBF76BFBFBFB664ADADBB
:10425000B6B6ADBFFF646DADB6AD6477BFBFBFFF8F
:10426000FF77BFBFBFFFFF7FBFBFBFFFF6BFB7ADC9
:10427000F6FFFFA4ADFFFFFFFFFFFFFFFFFFFFFF04
:10428000FFFFF6A4005B5200000000BFBFAD5B64FF
:10429000BFB6ADADBFFFBFFFFFFFFFBF64FFFFBFF6
:1042A000B6765BFFBFBF5B0000FF5C000000000054
:1042B0000000000000000000000000BFBF645C5C64
:1042C000006E5C654900006D5B00000000000000AE
:1042D00000000000000000000000000000000000DE
:1042E00000000000000000000000000600040000C4
:1042F000000100020003000400050006000700089A
:104300000009000A000B000C000D000E000F001049
:104310000000001100120013001400150016000622
:1043200000030000001700180019001A001B001CF1
:10433000001D001E001F0020002100220023002479
:1043400000250026000000000002080008550408AF
:104350005A0000F8000990000A1E32050000FF47CD
:1043600043000000010002000300040005010001F9
:10437000010102010301040105020002010202021F
:104380000302040205030003010302030303040301
:1043900005040004010402040304040405050005E7
:1043A00001050205030504050506000601060206CF
:1043B00003060406050700070107020703070407B1
:1043C0000508000801080208030804080509000997
:1043D0000109020903090409050A000A010A020A7F
:1043E000030A040A050B000B010B020B030B040B61
:1043F000050C000C010C020C030C040C050D000D47
:10440000010D020D030D040D050E000E010E020E2E
:10441000030E040E050F000F010F020F030F040F10
:1044200005100010011002100310041005110011F6
:1044300001110211031104110512001201120212DE
:1044400003120412051300130113021303130413C0
:1044500005140014011402140314041405150015A6
:10446000011502150315041505160016011602168E
:104470000316041605170017011702170317041770
:104480000518001801180218031804180519001956
:104490000119021903190419051A001A011A021A3E
:1044A000031A041A051B001B011B021B031B041B20
:1044B000051C001C011C021C031C041C051D001D06
:1044C000011D021D031D041D051E001E011E021EEE
:1044D000031E041E051F001F011F021F031F041FD0
:1044E000050011241FBECFEFD0E1DEBFCDBF14BE4B
:1044F00088E10FB6F89480936000109260000FBEC0
:1045000011E0A0E0B1E0E6EEFAE902C005900D92FC
:10451000AE31B107D9F71CE0AEE1B1E001C01D92A8
:10452000A538B107E1F70E942A2B0E94CD4B0E94CB
:1045300021250E948B230C94714D0C9400008093D4
:10454000960B6093970B382F3A5F3093990B6093DB
:104550009A0B282F245F20939C0B60939D0B982F20
:104560009E5E90939F0B6093A00B8093A20B685F5D
:104570006093A30B3093A50B6093A60B2093A80B1D
:104580006093A90B9093AB0B6093AC0B0895CF9302
:10459000DF9380E00E94E624EC0190FF40C0809110
:1045A00022019091230190FD3AC0809120019091C9
:1045B000210101969093210180932001039721F41A
:1045C00010922101109220018091200190912101EF
:1045D000009739F442EF52E060E280E00E948031BF
:1045E00011C08130910591F44EEA52E060E280E022
:1045F0000E94803140E85BE361E270E081E090E09E
:104600000E948D3283E08093020104C0029711F46E
:10461000109202018091020180580E94474CC0FF15
:1046200007C0809100018A3818F48F5F80930001E1
:10463000C1FF07C080910001882319F08150809349
:104640000001C4FF0EC080911E018F5F80931E0188
:10465000803C10F010921E01809100018F5F8093CA
:104660000001C5FF0FC080911E01815080931E0183
:104670008F3F19F48FEB80931E01809100018150D0
:1046800080930001C7FF0AC080911F018150809371
:104690001F0180910101815080930101C6FF0AC072
:1046A00080911F018F5F80931F01809101018F5FB7
:1046B00080930101D1FF21C020E040E050E060E0A4
:1046C00080E00E94482620E040E050E060E081E089
:1046D0000E94482620E040E050E060E082E00E9436
:1046E000482620E040E050E060E083E00E94482659
:1046F00080E00E94E624892BD9F760911F01809108
:104700001E010E94AD31D0932301C093220180E0AD
:10471000DF91CF9108952F923F925F926F927F9297
:104720008F929F92AF92BF92CF92DF92EF92FF92C1
:104730000F931F93DF93CF93CDB7DEB7C058D04010
:104740000FB6F894DEBF0FBECDBF86EE94E30E9495
:10475000424C86E393E00E94174C8DEB0E94CA4BBB
:104760000E94A34B8091020180580E94474C40E771
:1047700050E060E080E00E94803142EF52E060E271
:1047800080E00E94803146E45BE36BE170E082E010
:1047900090E00E948D3249E55BE36CE170E082E0DD
:1047A00090E00E948D324CE65BE36EE170E080E0C9
:1047B00090E00E948D321092950BE0EBFBE081E0DF
:1047C000808333969BE0E53FF907D1F788E180933A
:1047D000980B89E180939B0B8AE180939E0B8BE180
:1047E0008093A10B8CE18093A40B8DE18093A70BA8
:1047F0008EE18093AA0B8FE18093AD0B6091010154
:10480000809100010E949F2280E190E00E94A04CD4
:104810007AE0C72ED12CCC0EDD1E6AE4E62EF12CF8
:10482000EC0EFD1E5AE2A52EB12CAC0EBD1E8E0163
:1048300006591F4F88248A949924939441E2642E48
:10484000712C6C0E7D1E0E949B4C6EE670E00E94E7
:10485000B74C8E5FF60180830E949B4C60E170E054
:104860000E94B74C883018F4F801908202C0F80119
:1048700080820E949B4C64EB70E00E94B74C8E5F7C
:10488000F50180830E949B4C60E170E00E94B74C70
:104890008A3018F4F701908202C0F70180820894F0
:1048A000C11CD11C0894E11CF11C0894A11CB11C72
:1048B0000F5F1F4FC614D70431F636E0832E912CBC
:1048C0008C0E9D1E26E4A22EB12CAC0EBD1E96E6CB
:1048D000C92ED12CCC0EDD1E86E2E82EF12CEC0E7A
:1048E000FD1E552453940FEF81E090E00E94E633C3
:1048F0009401D50162EA7BE01601A7018C91F901D0
:104900001081180F10831E3720F0813039F40C937A
:1049100005C01D3018F48F3F09F45C92F1019081BD
:10492000FA018081890F80838C3B28F0913049F413
:10493000F101008306C0843020F49F3F11F4F1019F
:104940005082FB01108381832F5F3F4F11966D5F73
:104950007F4F0894211C311C4F5F5F4F2615370590
:1049600069F60E94C72260910101809100010E94B6
:104970009F2245E95BE36CE070E085E090E00E94F7
:104980008D3240911E016CE070E089E090E00E9461
:10499000FA3248E95BE36CE070E08CE090E00E9462
:1049A0008D3240911F016CE070E080E190E00E9448
:1049B000FA329ACF28E088E190E00FB6F894A895F3
:1049C000809360000FBE209360000895882329F42F
:1049D00080910B0C90910C0C04C080910D0C909167
:1049E0000E0C909325018093240140912401509155
:1049F00025014F3F510519F1CA0180709370805015
:104A00009340E9F4CA018870987088509840B9F4CE
:104A100080910B0C90910C0C892B31F080910D0C36
:104A200090910E0C892BA1F728E088E190E00FB659
:104A3000F894A895809360000FBE20936000CA018F
:104A400008950F931F938FE593E40E94BA250BE915
:104A50001BE3C8010E94174CC8010E94124C0E941F
:104A6000A34B8FE090E00E94E63341E06FEF80E0DF
:104A70000E9404290BEE12E4A8016CE088E00E9479
:104A8000993383E090E00E94E6334FE153E46CE019
:104A900088E00E94993382E090E00E94E633A8010A
:104AA0006CE088E00E94993388E290E00E94E6334F
:104AB0000E94A34B84E190E00E94E6331F910F9186
:104AC000089590E025E130E0829FF001839FF00D92
:104AD000929FF00D1124EE5DF34F6187089560936E
:104AE0004C03089590E025E130E0829FF001839F20
:104AF000F00D929FF00D1124EE5DF34F128611829E
:104B0000089590E025E130E0829FF001839FF00D51
:104B1000929FF00D1124EE5DF34F81E0828B08959A
:104B200090E025E130E0829FF001839FF00D929F9D
:104B3000F00D1124EE5DF34F6087089590E025E1BC
:104B400030E0829FF001839FF00D929FF00D1124C1
:104B5000EE5DF34F6483089590E025E130E0829F9D
:104B6000F001839FF00D929FF00D1124EE5DF34F45
:104B7000658308959093790C8093780C10922601A8
:104B8000E2E2FCE021E08FEF98E120831782868348
:104B9000138680871182958375963CE0E637F3078C
:104BA000A1F708951092230C1092380C10924D0C1E
:104BB0001092620C01969093810C8093800C9093DC
:104BC000210C8093200C9093840C8093830C109282
:104BD0007F0C10927E0C1092770C1092760C109233
:104BE0007A0C81E08093260110927D0C10927C0C4F
:104BF00008958091200C9091210C0E94D225089557
:104C000080912B0C87FD03C08AEF80932B0C809141
:104C1000400C87FD03C08AEF8093400C8091550CB7
:104C200087FD03C08AEF8093550C80916A0C87FD45
:104C300003C08AEF80936A0C10922601089581E0E8
:104C4000809326010895DC01ED91FC911197AF014D
:104C50004F5F5F4F11965C934E93E4912E2F30E09F
:104C6000E7FF13C02F7730703695322F2227379504
:104C70002795FA014F5F5F4FE4918E2F8F77280FB2
:104C8000311DE7FDF1CF4D935C93C901089508955F
:104C90000F931F93CF93DF93182F062FEA018330D2
:104CA00049F481E091E090934E0380934D0320936B
:104CB0004C0310C0622F0E941F2A812F90E0FC013C
:104CC000EE0FFF1FE80FF91FEE0FFF1FE75CFC4F11
:104CD000D283C183212F30E085E190E0289FF0014D
:104CE000299FF00D389FF00D1124EE5DF34F81E008
:104CF00082870783DF91CF911F910F9108950E94C2
:104D00001F2A0895EF92FF920F931F93CF93DF9383
:104D1000182F062FF42EE22EC82FD0E085E190E068
:104D2000C89FF001C99FF00DD89FF00D1124EE5DD2
:104D3000F34F8285882321F08181882309F077C091
:104D4000EE2091F485E190E0C89FF001C99FF00D3D
:104D5000D89FF00D1124EE5DF34F128A81858823D0
:104D600009F065C0178263C0133059F481E091E007
:104D700090934E0380934D0381E080934C030F2D5D
:104D800008C060E0812F0E941F2A6F2D812F0E9492
:104D9000002A0F3799F485E190E0C89FF001C99F80
:104DA000F00DD89FF00D1124EE5DF34F80917C0C37
:104DB00086878DE79CE0948B838B20C0802F90E0CA
:104DC000880F991FE091780CF091790CE80FF91F8A
:104DD000259134912F5F3F4FF901449185E190E097
:104DE000C89FF001C99FF00DD89FF00D1124EE5D12
:104DF000F34F46872F5F3F4F348B238B85E190E045
:104E0000C89FF001C99FF00DD89FF00D1124EE5DF1
:104E1000F34F17861186038711828FEF8087E78211
:104E2000F282108A81E08287128A118A1482DF91CD
:104E3000CF911F910F91FF90EF900895CF92DF9245
:104E4000FF920F931F93CF93DF93EAE2FCE08181FF
:104E5000282F332727FD30958081280F311D2F3FC4
:104E6000310519F014F02FEF30E0C90137FF02C00F
:104E700080E090E0808375964CE0EE37F40739F7D8
:104E800080912601882309F0D9C0F5C0E091800CFB
:104E9000F091810C9F012F5F3F4F3093810C209345
:104EA000800C44914F3F69F5A9014F5F5F4F5093CC
:104EB000810C4093800CF90184918F3219F4109287
:104EC0002601CAC0863009F0AAC0FA013196CF0186
:104ED00001969093810C8093800CE491E33529F442
:104EE0009093840C8093830C9AC0E53409F097C0AA
:104EF0008091830C9091840C9093810C8093800C12
:104F00008EC047FF02C040937A0C542F5F70842FED
:104F100090E0807F9070803B910529F1803C910565
:104F200029F18039910509F038C0C9010196F901CC
:104F3000449101969093810C8093800C0197FC0121
:104F40002491852F90E08C9FF0018D9FF00D9C9F08
:104F5000F00D1124EE5DF34F8081882309F45FC0CA
:104F6000220F638545C02E5F3F4F48C02F5F3F4FE4
:104F70003093810C2093800C21503040F901249112
:104F8000852F90E08C9FF0018D9FF00D9C9FF00D80
:104F90001124EE5DF34F238742C080917A0C582F85
:104FA0005F7090E0807F9070803B910529F1803C9C
:104FB000910549F18039910591F52F5F3F4F30936D
:104FC000810C2093800C21503040F9012491852FD1
:104FD00090E08C9FD0018D9FB00D9C9FB00D11244F
:104FE000AE5DB34F8C918823D1F0220F1B966C914C
:104FF000852F0E94822613C02F5F3F4F3093810C74
:105000002093800C0CC0852F90E08C9FF0018D9F29
:10501000F00D9C9FF00D1124EE5DF34F438780E867
:105020009CE00E9423269695879590937F0C809311
:105030007E0C1092770C1092760C02C0C5E1D0E085
:105040006091760C7091770C80917E0C90917F0C22
:105050006817790709F41ACF6F5F7F4F7093770C49
:105060006093760C80917C0C90917D0C01969093CE
:105070007D0C80937C0C09E313E0C3E2DCE0FF24A9
:105080008FEFC82ED12C8989882309F05EC08A89C8
:105090009B89892B09F456C09E858D85981708F049
:1050A0004CC050C08A852A893B898F37E9F4D901E1
:1050B0008D91BB8BAA8B8F3F01F1F9016181119614
:1050C000BB8BAA8BE82FF0E0EE0FFF1FED5FFE4FCA
:1050D0000190F081E02D8F2D0995EA89FB8981915E
:1050E0008D87FB8BEA8B28C0A9014F5F5F4F5B8BDD
:1050F0004A8BF90184918F3F21F418821B8A1A8A06
:1051000021C04F5F5F4F5B8B4A8B41505040FA018B
:105110006491E82FF0E0EE0FFF1FED5FFE4F01906E
:10512000F081E02D8F2D0995EA89FB893196FB8B63
:10513000EA8B3197E491ED871E869E858D859817C1
:1051400009F4B0CF8E858F5F8E878985882319F407
:1051500020E030E047C08F858F3F11F08F5F8F8751
:105160009E819923C9F12F812223B1F18D8188235A
:1051700099F1899FC001112480509F4F892F992751
:1051800030E0AC01429FC001439F900D529F900DB3
:10519000112480509F4F292F33278B818823F1F0D2
:1051A000EA81F0E0E050F84AE491E058E89FC0015D
:1051B000112480509F4F892F9927F601E81BF90B86
:1051C000E29FC001E39F900DF29F900D112480504B
:1051D0009F4F292F332702C020E030E08A819C8135
:1051E000890F8A83F8012083F3940A5F1F4F659625
:1051F000F4E0FF1609F047CFDF91CF911F910F9197
:10520000FF90DF90CF9008951F93CF93DF93582F97
:1052100090E0880F991F2091780C3091790C280F1D
:10522000391FF90185919491DC011196FC0184915B
:10523000813011F413E01DC08091380C8823B1F047
:105240008091430C851711F4442381F480914D0C17
:10525000882371F08091580C851711F4442341F490
:105260009091470C80915C0C891710F411E001C0FB
:1052700012E0212F30E0FD01449185E190E0289F6C
:10528000E001299FD00D389FD00D1124CE5DD34F62
:105290004E871196BC8BAB8B1F8680E58A836F830C
:1052A0008FEF888719861A8A188A21E02A87198A37
:1052B0005C8729831C82133049F481E091E090934C
:1052C0004E0380934D0320934C0308C060E5812F6B
:1052D0000E94002A6989812F0E941F2ADF91CF91A5
:1052E0001F910895FF920F931F93082FF62E0E948F
:1052F000002A10E085E190E0089FF001099FF00D81
:10530000189FF00D1124EE5DF34FF2821F910F9163
:10531000FF900895962F482F50E025E130E0429FFE
:10532000F001439FF00D529FF00D1124EE5DF34FFD
:105330006281691B62830E94002A0895482F50E011
:1053400025E130E0429FF001439FF00D529FF00DA8
:105350001124EE5DF34F9281690F62830E94002A4F
:1053600008950000000000000000000000000000A0
:10537000000000000000000000000000000000002D
:10538000000000000000000000000000000000001D
:10539000000000000000000000000000000000000D
:1053A00000000000000000000000000000000000FD
:1053B00000000000000000000000000000000000ED
:1053C00000000000000000000000000000000000DD
:1053D00000000000000000000000000000000000CD
:1053E00000000000000000000000000000000000BD
:1053F00000000000000000000000000000000000AD
:1054000099277727833008F00895E0E0F2E6660FE9
:10541000771FE60FF71FA591B491E9E3F3E026E0CB
:10542000289FE00DF11DA183B2831124089590916E
:105430004C039170880F892B80934C030895992712
:105440007727E9E3F3E026E0289FE00DF11D6E3FAA
:1054500031F460914C036E7F60934C030BC06F3F3F
:1054600031F460914C036E6F60934C0303C078E598
:10547000760F75831124089599277727E9E3F3E0E0
:1054800026E0289FE00DF11D6083112408952F93DD
:105490003F934F935F936F937F938F939F93AF93BC
:1054A000BF93789411240E94C3310E94A14A0E94A4
:1054B0001E272F923F924F925F926F927F928F9210
:1054C0009F92AF92BF92CF92DF92EF92FF920F9393
:1054D0001F93CF93DF9300903603002019F4AAE2C4
:1054E000B1E002C0AFE2B2E001E000260092360374
:1054F00002E00093370320903A0330903B03409042
:105500003D0350903E0360903C031091390370902E
:1055100040038090410390904203A0904303B090D9
:10552000440320913F03C0904603D0904703E0908E
:105530004903F0904A03009148033091450350918C
:105540004B0360914D0370914E0380914F039FEF89
:10555000620C431CF2014491410300240008C12D58
:10556000D02D970CA81CF50144914203002400089B
:10557000C10DD01D0C0DED1CF70144914303002417
:105580000008C10DD01D8A956AF440914C03842F08
:105590008695062E0694062600FA7695679576F986
:1055A00040FF66F940E860FD4FE74503002400082E
:1055B000C10DD01DD595C7950024C038D0050CF07D
:1055C000CFE70A94C038D0050CF4C0E8CD939A9583
:1055D00009F0BECF409137034A954093370396E0D8
:1055E00009F0B6CF60923C0340923D039092420393
:1055F000A092430300934803E092490360934D0354
:1056000070934E0380934F03DF91CF911F910F91C1
:10561000FF90EF90DF90CF90BF90AF909F908F90D2
:105620007F906F905F904F903F902F90992780913F
:10563000000C77276091010C11240E944726BF912E
:10564000AF919F918F917F916F915F914F913F911A
:105650002F910895AAE2B1E08AE092E000E00D9374
:105660000197E9F7AAE2B1E0A0933403B0933503C0
:1056700000270093360368E560933E03609344037C
:1056800060934A0361E060934D0360934E0361E0D1
:1056900060934C0366276093390360933F036093E4
:1056A000450360934B0360933A0360933B0360931D
:1056B0003C0360933D036093400360934103609318
:1056C00042036093430360934603609347036093F0
:1056D00048036093490311240895E0913403F09145
:1056E0003503019100580093B30003E0E433F00761
:1056F0000AE211E008F0F801E0933403F093350377
:1057000008950C94832B0C94852B0F931F932ABD23
:10571000E0913403F0913503019100580093B300F8
:1057200003E0E433F00710F40000000010F0EAE2B8
:10573000F1E0E0933403F0933503C895C895C8951C
:10574000C895C895C8950000000000002AB51F91B3
:105750000F9108950000E091010CE0FFD6CFE1E148
:10576000EA95F1F700000000089500000000000035
:105770000000000000000000000000000000000029
:105780000000000000000000000000000000000019
:105790000000000000000000000000000000000009
:1057A00000000000000000000000000000000000F9
:1057B00000000000000000000000000000000000E9
:1057C00000000000000000000000000000000000D9
:1057D00000000000000000000000000000000000C9
:1057E00000000000000000000000000000000000B9
:1057F00000000000000000000000000000000000A9
:10580000000306090C101316191C1F2225282B2E25
:10581000313336393C3F414447494C4E515355583A
:105820005A5C5E60626466686A6B6D6F70717374F7
:10583000757678797A7A7B7C7D7D7E7E7E7F7F7FB0
:105840007F7F7F7F7E7E7E7D7D7C7B7A7A79787696
:1058500075747371706F6D6B6A68666462605E5CAC
:105860005A585553514E4C494744413F3C393633C1
:10587000312E2B2825221F1C191613100C09060384
:1058800000FDFAF7F4F0EDEAE7E4E1DEDBD8D5D28B
:10589000CFCDCAC7C4C1BFBCB9B7B4B2AFADABA856
:1058A000A6A4A2A09E9C9A9896959391908F8D8C79
:1058B0008B8A8887868685848383828282818181A0
:1058C0008181818182828283838485868687888A9A
:1058D0008B8C8D8F9091939596989A9C9EA0A2A464
:1058E000A6A8ABADAFB2B4B7B9BCBFC1C4C7CACD2F
:1058F000CFD2D5D8DBDEE1E4E7EAEDF0F4F7FAFD4C
:10590000808182838485868788898A8B8C8D8E8F1F
:10591000909192939495969798999A9B9C9D9E9F0F
:10592000A0A1A2A3A4A5A6A7A8A9AAABACADAEAFFF
:10593000B0B1B2B3B4B5B6B7B8B9BABBBCBDBEBFEF
:10594000C0C1C2C3C4C5C6C7C8C9CACBCCCDCECFDF
:10595000D0D1D2D3D4D5D6D7D8D9DADBDCDDDEDFCF
:10596000E0E1E2E3E4E5E6E7E8E9EAEBECEDEEEFBF
:10597000F0F1F2F3F4F5F6F7F8F9FAFBFCFDFEFFAF
:10598000000102030405060708090A0B0C0D0E0F9F
:10599000101112131415161718191A1B1C1D1E1F8F
:1059A000202122232425262728292A2B2C2D2E2F7F
:1059B000303132333435363738393A3B3C3D3E3F6F
:1059C000404142434445464748494A4B4C4D4E4F5F
:1059D000505152535455565758595A5B5C5D5E5F4F
:1059E000606162636465666768696A6B6C6D6E6F3F
:1059F000707172737475767778797A7B7C7D7E7F2F
:105A000000020406080A0C0E10121416181A1C1EA6
:105A100020222426282A2C2E30323436383A3C3E96
:105A200040424446484A4C4E50525456585A5C5E86
:105A300060626466686A6C6E70727476787A7C7E76
:105A40007F7D7B79777573716F6D6B696765636156
:105A50005F5D5B59575553514F4D4B494745434146
:105A60003F3D3B39373533312F2D2B292725232136
:105A70001F1D1B19171513110F0D0B090705030126
:105A8000FFFDFBF9F7F5F3F1EFEDEBE9E7E5E3E116
:105A9000DFDDDBD9D7D5D3D1CFCDCBC9C7C5C3C106
:105AA000BFBDBBB9B7B5B3B1AFADABA9A7A5A3A1F6
:105AB0009F9D9B99979593918F8D8B8987858381E6
:105AC00080828486888A8C8E90929496989A9C9EE6
:105AD000A0A2A4A6A8AAACAEB0B2B4B6B8BABCBED6
:105AE000C0C2C4C6C8CACCCED0D2D4D6D8DADCDEC6
:105AF000E0E2E4E6E8EAECEEF0F2F4F6F8FAFCFEB6
:105B00007F7F7F7F7F7F7F7F7F7F7F7F7F7F7F7FA5
:105B10007F7F7F7F7F7F7F7F7F7F7F7F7F7F7F7F95
:105B20007F7F7F7F7F7F7F7F7F7F7F7F7F7F7F7F85
:105B30007F7F7F7F7F7F7F7F7F7F7F7F7F7F7F7F75
:105E00000309131E28313A40464C5054585B5E61DA
:105E1000636567696B6C6E6F70717273747576779A
:105E2000777879797A7A7B7B7C7C7C7D7D7D7E7EC0
:105E30007E7E7F7F7F7F7F7F7F7F7F7F7F7F7F7F74
:105E40007F7F7F7F7F7F7F7F7F7F7F7F7F7E7E7E65
:105E50007E7D7D7D7C7C7C7B7B7A7A797978777797
:105E6000767574737271706F6E6C6B696765636160
:105E70005E5B5854504C46403A31281E13090300CB
:105E8000C6CCD5DBDFE3E5E7E9EAEBECEDEEEFEFDF
:105E9000F0F0F0F1F1F1F1F2F2F2F2F2F2F2F2F3EB
:105EA000F3F3F3F3F3F3F3F3F3F3F3F3F3F3F3F3C2
:105EB000F3F3F3F3F3F3F3F3F3F3F3F3F3F3F3F3B2
:105EC000F3F3F3F3F3F3F3F3F3F3F3F3F3F3F3F3A2
:105ED000F3F3F3F3F3F3F3F3F3F3F3F3F3F3F3F392
:105EE000F2F2F2F2F2F2F2F2F1F1F1F1F0F0F0EF9F
:105EF000EFEEEDECEBEAE9E7E5E3DFDBD5CCC6005E
:105F000000283D42302D2C2B2C2D2E2F30323335B6
:105F100037393B3D3F414345484A4C4E5053555716
:105F2000595B5D5F61636567696B6C6E70717374FB
:105F3000757778797A7B7C7D7D7E7E7F7F7F7F7FA2
:105F40007F7F7F7F7F7F7E7E7D7D7C7B7A79787788
:105F500075747371706E6C6B69676563615F5D5BAF
:105F600059575553504E4C4A484543413F3D3B39A4
:105F700037353332302F2E2D2C2B2C2D30423D280F
:105F800000E9E5FED4D7D7D7D6D4D2D0CECCCAC874
:105F9000C6C3C1BFBDBAB8B6B4B1AFADABA9A7A5B2
:105FA000A3A19F9E9C9A999795949391908F8D8C85
:105FB0008B8A898888878685858484848383838384
:105FC0008383838383848484858586878888898A7C
:105FD0008B8C8D8F909193949597999A9C9E9FA16D
:105FE000A3A5A7A9ABADAFB1B4B6B8BABDBFC1C385
:105FF000C6C8CACCCED0D2D4D6D7D7D7D4FEE5E93E
:10600000F9F8F9F5EBE1DDDEE0E2E4E5E6E5E4E20E
:10601000DED9D2CAC1B7ACA299918A868381808029
:106020008182838586888A8C8D8F909293959697AE
:1060300098999A9B9B9C9D9D9D9E9E9E9F9F9F9F96
:106040009F9F9F9E9E9E9D9D9D9C9B9B9A9998978E
:1060500096959392908F8D8C8A8886858382818095
:10606000808183868A9199A2ACB7C1CAD2D9DEE277
:10607000E4E5E6E5E4E2E0DEDDE1EBF5F9F8F90080
:106080000708070B151F2322201E1C1B1A1B1C1E92
:1060900022272E363F49545E676F767A7E7F7F7F58
:1060A0007F7E7D7B7A7876747371706E6D6B6A69B2
:1060B00068676665656464636362626261616161A9
:1060C0006161616262626363636465656667686992
:1060D0006A6B6D6E7071737476787A7B7D7E7F7F6C
:1060E0007F7F7E7A766F675E54493F362E27221E69
:1060F0001C1B1A1B1C1E2022231F150B0708070040
:106100001F313D444E5354565A5F64696E7476791C
:106110007C7F7F7F7F7F7F7F7F7F7F7F7F7F7F7F92
:106120007F7F7F7F7F7F7F7F7F7F7F7F7F7F7F7F7F
:106130007F7F7F7F7F7F7F7F7F7F7F7F7F7F7F7F6F
:106140007F7F7F7F7F7F7F7F7F7F7F7F7F7F7F7F5F
:106150007F7F7F7F7F7F7F7F7F7F7F7F7F7F7F7F4F
:106160007F7F7F7F7F7F7F7F7F7F7F7F7F7F7F7F3F
:106170007F7F7F7F7F7F7F7F7F7F7F7C7871684C91
:106180002C1C120C0A0B0A05FDF3E9DFD4CAC0B7B8
:10619000AEA69E97918B868582808080808080804D
:1061A00080808080808080808080808080808080EF
:1061B00080808080808080808080808080808080DF
:1061C00080808080808080808080808080808080CF
:1061D00080808080808080808080808080808080BF
:1061E00080808080808080808080808080808080AF
:1061F000808080808087919DACC4CBD4DDF2FAFA98
:1062000022002400260028002B002D00300033003F
:10621000360039003D004000440048004C00510069
:1062200056005B00600066006C007300790081001E
:10623000880090009900A200AC00B600C100CC001C
:10624000D800E500F30001011001210132014401F1
:1062500057016C0181019801B001CA01E5010202F8
:106260002102410264028802AE02D7020303300316
:1062700061039403CB03050442048304C70410059F
:106280005D05AF0505066106C206290796070908E0
:10629000830805098E09200ABA0A5D0B0A0CC10C95
:1062A000840D510E2B0F121007110A121D134014EA
:1062B0007415BA1614188319071BA31C571E242023
:1062C0000E22142439267F28E82A752D293006331A
:1062D0000F364539AD3C49401B442848734CFE50AD
:1062E000CF55EA5A51600C661D6C8B725A799280B8
:1062F00037885090E598FDA19FABD3B5A3C00000AF
:106300001F93CF93DF93FA01549131961491C52FC7
:10631000D0E09F012F5F3F4F70E095E0660F771F41
:106320009A95E1F7680F711D40E00BC084918D9341
:106330009F5F31969517D0F34F5F2C0F3D1F605E26
:106340007F4F411730F4DB01A05ABC4FF90190E0B8
:10635000F1CFDF91CF911F910895803C88F4282FD1
:1063600030E0220F331FC9018F599C4BFC018491EF
:106370002E593C4BF90194918093FE0B9093FD0BA9
:106380006093FF0B0895CF92DF92EF92FF921F93DD
:10639000CF93DF938091C00787FF0AC090E08F7092
:1063A0009070009729F00196880F880F880F01C020
:1063B00088E0E3E5F8E010821182128213823496BD
:1063C0009BE0E339F907B9F7C6E9DBE061E0C82EE5
:1063D000DD2419819881812F8150873D08F055C0B7
:1063E000992309F452C09A3808F04FC0712F7850A1
:1063F00040E050E0E12EFF24942F9A012E0D3F1D26
:106400002C153D05E4F1283D3105CCF5272F30E072
:10641000D901AA0FBB1FAA0FBB1FAD5AB74F8C9152
:10642000882331F49295990F907E960F9C9327C004
:1064300011968C911197882339F49295990F907E3B
:10644000960F11969C931BC0F901EE0FFF1FEE0FE4
:10645000FF1FEB5AF74F8081882331F49295990FF3
:10646000907E960F90830BC013968C911397882380
:1064700031F49295990F907E960F13969C934F5FEF
:106480005F4F7F5F711709F0B7CF6F5F2396603260
:1064900009F09FCFDF91CF911F91FF90EF90DF9098
:1064A000CF9008958F929F92AF92BF92CF92DF923A
:1064B000EF92FF920F931F93CF93DF93882E962E28
:1064C0005A016901F02E00E010E080EEF80E0CC0D9
:1064D0004F2D6E2D882D8C0F0E94BB4B2196CA1517
:1064E000DB05B4F30F5F1F4F0C151D052CF4C0E046
:1064F000D0E0E02EE90CF3CFDF91CF911F910F9107
:10650000FF90EF90DF90CF90BF90AF909F908F90D3
:10651000089540520E94BB4B0895FF920F931F9322
:10652000CF93DF938C01F62EEA01FE014491219670
:10653000442349F0802F0F5F1F4F4F7740526F2D3C
:106540000E94BB4BF2CFDF91CF911F910F91FF9033
:106550000895FF920F931F93182F062FF42E429544
:106560004F704A3010F4405F01C0495E602F812FA8
:106570000E94BB4B4F2D4F70812F8F5F4A3010F41C
:10658000405F01C0495E602F0E94BB4B1F910F917D
:10659000FF900895FF920F931F93F82E162F042F4C
:1065A000452F0E94A932402F612F8F2D8E5F0E94B0
:1065B000A9321F910F91FF900895EF92FF920F93D0
:1065C0001F93F62E042F182FF8E0EF2EE80E07FF8A
:1065D00002C041E101C040E16F2D812F0E94BB4B01
:1065E0001F5F1E1511F0000FF2CF1F910F91FF904A
:1065F000EF900895FF920F931F93CF93DF93F62EA2
:10660000042FEC0110E0002311F4112339F4802F42
:106610006AE00E94AB4C905F492F01C040E06F2DB3
:106620008C2F0E94BB4B1F5F2197133031F0802FBE
:106630006AE00E94AB4C082FE6CFDF91CF911F910B
:106640000F91FF900895CF92DF92EF92FF920F93F8
:106650001F93CF93DF93C62E79018A01EC01DD24CD
:10666000E114F1040105110511F4DD2059F4C8010C
:10667000B7012AE030E040E050E00E94CA4C462FCB
:10668000405F01C040E06C2D8C2F0E94BB4BD39427
:10669000219786E0D81669F0C801B7012AE030E0FA
:1066A00040E050E00E94CA4CC901DA017C018D0132
:1066B000D7CFDF91CF911F910F91FF90EF90DF9097
:1066C000CF9008957F928F929F92AF92BF92CF9278
:1066D000DF92EF92FF920F931F93CF93DF93782E69
:1066E000862E5A016901780100E010E00CC0A70174
:1066F000692D872D8C0F0E94AD4B2196CA15DB05A5
:10670000B4F30F5F1F4F0C151D052CF4C0E0D0E053
:10671000902E980CF3CFDF91CF911F910F91FF90A6
:10672000EF90DF90CF90BF90AF909F908F907F9031
:1067300008957F928F929F92AF92BF92CF92DF92F5
:10674000EF92FF920F931F93CF93DF93782E862EB5
:10675000EA01FA01C590D490FA013296A590B4905E
:1067600000E016C0FC01EE0DFF1D3296EE0FFF1F7C
:10677000EC0FFD1F45915491692D812F870D0E94CB
:10678000AD4B1F5F812F90E08C159D055CF30F5F73
:10679000802F90E08A159B055CF48C9D70018D9D87
:1067A000F00C9C9DF00C112410E0902E980CEACF78
:1067B000DF91CF911F910F91FF90EF90DF90CF90DD
:1067C000BF90AF909F908F907F9008950F931F93ED
:1067D000CF93DF938C01C0E0D0E007C00E94214C32
:1067E0008823E1F30E94244C2196C017D107B4F30B
:1067F000DF91CF911F910F910895614B6B4B794BB6
:106800008F4A5F35DC385B3CDA3F5A43DB46E8EDC4
:10681000C8950000EA95E1F7C0E6D3E000240091B6
:10682000FE0BC00FD01DCABDDBBD2091C007277075
:10683000022F220F220F220F7091FF0B720F672F72
:10684000262E677026942694269410E2219EC00D71
:10685000D11DC093C107D093C207EE24A0E6B7E0D4
:1068600000242011ED012011F72E2011962E201169
:1068700066272011E39420E8201B00EDA02EA3E55D
:10688000B8E041D000C000C03D01A3EFBBE00EEF77
:1068900014E0ED91FD910193019301930193019314
:1068A00001931A95B1F7D301AA9401F173956395F9
:1068B00000C0683021F008E00A95F1F7E2CF6627C2
:1068C000A0960AB41BB42090C1073090C20723954C
:1068D0000BF4E1010BF4692D0BF47F2D0BF4EE2486
:1068E00044247030E40409F4E001CBCF05E00A95BC
:1068F000F1F700000E94524BE1E0E093020CE2E06D
:10690000E0933600089528980E946D2B2F931E0166
:10691000C090FB0BD090FC0B80E323E036E099277E
:106920000D91102F0F71129516951770C3E9DBE0CA
:10693000029FC00DD11D4880F6010A81089FE00D1D
:10694000F11D139FE00DF11DC3ECD7E0C40DD91F5D
:10695000C093F30BD093F40B059009920590099224
:106960000590099205900992059009920590099267
:106970000D91102F0F71129516951770C3E9DBE07A
:10698000029FC00DD11D4880F6010A81089FE00DCD
:10699000F11D139FE00DF11DC3ECD7E0C40DC093B2
:1069A000F50BD91F289AD093F60B05900992059004
:1069B0000992059009920590099205900992059017
:1069C00009920D91102F0F71129516951770C3E94A
:1069D000DBE0029FC00DD11D4880F6010A81089FAF
:1069E000E00DF11D139FE00DF11DC3ECD7E0C40DC8
:1069F000D91FC093F70BD093F80B0590099205901F
:106A000009920590099205900992059009920590C6
:106A100009920D91102F0F71129516951770C3E9F9
:106A2000DBE0029FC00DD11D4880F6010A81089F5E
:106A3000E00DF11D139FE00DF11DC3ECD7E0C40D77
:106A4000D91FC093F90BD093FA0B059009920590CA
:106A50000992059009920590099205900992059076
:106A60000992E101E091010CEA95E093010C3D01EE
:106A7000DE013C2F307E1EEFC9ECD7E04090040CC5
:106A80005090050C26E0629FC001E2E0F8E680909D
:106A9000FD0B40E0E4128824880C1124E80DF11D60
:106AA00005901490F00186944C9120E3429FA395A9
:106AB000AF71A32B040C151C080E191E0994F001CC
:106AC000C895C895C895C8950591D990D1120D2D36
:106AD00008B94C910591D990D1120D2D08B9429F5A
:106AE0000591D990D1120D2D08B9040C151C0591F2
:106AF000D990D1120D2D08B9080E191E0591D99003
:106B0000D1120D2D08B9A395AF710591D990D1126D
:106B10000D2D08B9A32BF0010591D990D1120D2D9F
:106B200008B94C910591D990D1120D2D08B9429F09
:106B30000591D990D1120D2D08B9040C151C0591A1
:106B4000D990D1120D2D08B9080E191E0591D990B2
:106B5000D1120D2D08B9A395AF710591D990D1121D
:106B60000D2D08B9A32BF0010591D990D1120D2D4F
:106B700008B94C910591D990D1120D2D08B9429FB9
:106B80000591D990D1120D2D08B9040C151C059151
:106B9000D990D1120D2D08B9080E191E0591D99062
:106BA000D1120D2D08B9A395AF710591D990D112CD
:106BB0000D2D08B9A32BF0010591D990D1120D2DFF
:106BC00008B94C910591D990D1120D2D08B9429F69
:106BD0000591D990D1120D2D08B9040C151C059101
:106BE000D990D1120D2D08B9080E191E0591D99012
:106BF000D1120D2D08B9A395AF710591D990D1127D
:106C00000D2D08B9A32BF0010591D990D1120D2DAE
:106C100008B94C910591D990D1120D2D08B9429F18
:106C20000591D990D1120D2D08B9040C151C0591B0
:106C3000D990D1120D2D08B9080E191E0591D990C1
:106C4000D1120D2D08B9A395AF710591D990D1122C
:106C50000D2D08B9A32BF0010591D990D1120D2D5E
:106C600008B94C910591D990D1120D2D08B9429FC8
:106C70000591D990D1120D2D08B9040C151C059160
:106C8000D990D1120D2D08B9080E191E0591D99071
:106C9000D1120D2D08B9A395AF710591D990D112DC
:106CA0000D2D08B9A32BF0010591D990D1120D2D0E
:106CB00008B94C910591D990D1120D2D08B9429F78
:106CC0000591D990D1120D2D08B9040C151C059110
:106CD000D990D1120D2D08B9080E191E0591D99021
:106CE000D1120D2D08B9A395AF710591D990D1128C
:106CF0000D2D08B9A32BF0010591D990D1120D2DBE
:106D000008B94C910591D990D1120D2D08B9429F27
:106D10000591D990D1120D2D08B9040C151C0591BF
:106D2000D990D1120D2D08B9080E191E0591D990D0
:106D3000D1120D2D08B9A395AF710591D990D1123B
:106D40000D2D08B9A32BF0010591D990D1120D2D6D
:106D500008B94C910591D990D1120D2D08B9429FD7
:106D60000591D990D1120D2D08B9040C151C05916F
:106D7000D990D1120D2D08B9080E191E0591D99080
:106D8000D1120D2D08B9A395AF710591D990D112EB
:106D90000D2D08B9A32BF0010591D990D1120D2D1D
:106DA00008B94C910591D990D1120D2D08B9429F87
:106DB0000591D990D1120D2D08B9040C151C05911F
:106DC000D990D1120D2D08B9080E191E0591D99030
:106DD000D1120D2D08B9A395AF710591D990D1129B
:106DE0000D2D08B9A32BF0010591D990D1120D2DCD
:106DF00008B94C910591D990D1120D2D08B9429F37
:106E00000591D990D1120D2D08B9040C151C0591CE
:106E1000D990D1120D2D08B9080E191E0591D990DF
:106E2000D1120D2D08B9A395AF710591D990D1124A
:106E30000D2D08B9A32BF0010591D990D1120D2D7C
:106E400008B94C910591D990D1120D2D08B9429FE6
:106E50000591D990D1120D2D08B9040C151C05917E
:106E6000D990D1120D2D08B9080E191E0591D9908F
:106E7000D1120D2D08B9A395AF710591D990D112FA
:106E80000D2D08B9A32BF0010591D990D1120D2D2C
:106E900008B94C910591D990D1120D2D08B9429F96
:106EA0000591D990D1120D2D08B9040C151C05912E
:106EB000D990D1120D2D08B9080E191E0591D9903F
:106EC000D1120D2D08B9A395AF710591D990D112AA
:106ED0000D2D08B9A32BF0010591D990D1120D2DDC
:106EE00008B94C910591D990D1120D2D08B9429F46
:106EF0000591D990D1120D2D08B9040C151C0591DE
:106F0000D990D1120D2D08B9080E191E0591D990EE
:106F1000D1120D2D08B9A395AF710591D990D11259
:106F20000D2D08B9A32BF0010591D990D1120D2D8B
:106F300008B94C910591D990D1120D2D08B9429FF5
:106F40000591D990D1120D2D08B9040C151C05918D
:106F5000D990D1120D2D08B9080E191E0591D9909E
:106F6000D1120D2D08B9A395AF710591D990D11209
:106F70000D2D08B9A32BF0010591D990D1120D2D3B
:106F800008B94C910591D990D1120D2D08B9429FA5
:106F90000591D990D1120D2D08B9040C151C05913D
:106FA000D990D1120D2D08B9080E191E0591D9904E
:106FB000D1120D2D08B9A395AF710591D990D112B9
:106FC0000D2D08B9A32BF0010591D990D1120D2DEB
:106FD00008B94C910591D990D1120D2D08B9429F55
:106FE0000591D990D1120D2D08B9040C151C0591ED
:106FF000D990D1120D2D08B9080E191E0591D990FE
:10700000D1120D2D08B9A395AF710591D990D11268
:107010000D2D08B9A32BF0010591D990D1120D2D9A
:1070200008B94C910591D990D1120D2D08B9429F04
:107030000591D990D1120D2D08B9040C151C05919C
:10704000D990D1120D2D08B9080E191E0591D990AD
:10705000D1120D2D08B9A395AF710591D990D11218
:107060000D2D08B9A32BF0010591D990D1120D2D4A
:1070700008B94C910591D990D1120D2D08B9429FB4
:107080000591D990D1120D2D08B9040C151C05914C
:10709000D990D1120D2D08B9080E191E0591D9905D
:1070A000D1120D2D08B9A395AF710591D990D112C8
:1070B0000D2D08B9A32BF0010591D990D1120D2DFA
:1070C00008B94C910591D990D1120D2D08B9429F64
:1070D0000591D990D1120D2D08B9040C151C0591FC
:1070E000D990D1120D2D08B9080E191E0591D9900D
:1070F000D1120D2D08B9A395AF710591D990D11278
:107100000D2D08B9A32BF0010591D990D1120D2DA9
:1071100008B94C910591D990D1120D2D08B9429F13
:107120000591D990D1120D2D08B9040C151C0591AB
:10713000D990D1120D2D08B9080E191E0591D990BC
:10714000D1120D2D08B9A395AF710591D990D11227
:107150000D2D08B9A32BF0010591D990D1120D2D59
:1071600008B94C910591D990D1120D2D08B9429FC3
:107170000591D990D1120D2D08B9040C151C05915B
:10718000D990D1120D2D08B9080E191E0591D9906C
:10719000D1120D2D08B9A395AF710591D990D112D7
:1071A0000D2D08B9A32BF0012F910000000000273E
:1071B000E101D30108B90895F00131964C9100C066
:1071C00000C000C000C00591D990D1120D2D08B9A2
:1071D000429F0591D990D1120D2D08B9040C151CB0
:1071E0000591D990D1120D2D08B9080E191E0591DF
:1071F000D990D1120D2D08B9A395AF710591D990F1
:10720000D1120D2D08B9A32BF0010591D990D112FF
:107210000D2D08B94C910591D990D1120D2D08B9B9
:10722000429F0591D990D1120D2D08B9040C151C5F
:107230000591D990D1120D2D08B9080E191E05918E
:10724000D990D1120D2D08B9A395AF710591D990A0
:10725000D1120D2D08B9A32BF0010591D990D112AF
:107260000D2D08B94C910591D990D1120D2D08B969
:10727000429F0591D990D1120D2D08B9040C151C0F
:107280000591D990D1120D2D08B9080E191E05913E
:10729000D990D1120D2D08B9A395AF710591D99050
:1072A000D1120D2D08B9A32BF0010591D990D1125F
:1072B0000D2D08B94C910591D990D1120D2D08B919
:1072C000429F0591D990D1120D2D08B9040C151CBF
:1072D0000591D990D1120D2D08B9080E191E0591EE
:1072E000D990D1120D2D08B9A395AF710591D99000
:1072F000D1120D2D08B9A32BF0010591D990D1120F
:107300000D2D08B94C910591D990D1120D2D08B9C8
:10731000429F0591D990D1120D2D08B9040C151C6E
:107320000591D990D1120D2D08B9080E191E05919D
:10733000D990D1120D2D08B9A395AF710591D990AF
:10734000D1120D2D08B9A32BF0010591D990D112BE
:107350000D2D08B94C910591D990D1120D2D08B978
:10736000429F0591D990D1120D2D08B9040C151C1E
:107370000591D990D1120D2D08B9080E191E05914D
:10738000D990D1120D2D08B9A395AF710591D9905F
:10739000D1120D2D08B9A32BF0010591D990D1126E
:1073A0000D2D08B94C910591D990D1120D2D08B928
:1073B000429F0591D990D1120D2D08B9040C151CCE
:1073C0000591D990D1120D2D08B9080E191E0591FD
:1073D000D990D1120D2D08B9A395AF710591D9900F
:1073E000D1120D2D08B9A32BF0010591D990D1121E
:1073F0000D2D08B94C910591D990D1120D2D08B9D8
:10740000429F0591D990D1120D2D08B9040C151C7D
:107410000591D990D1120D2D08B9080E191E0591AC
:10742000D990D1120D2D08B9A395AF710591D990BE
:10743000D1120D2D08B9A32BF0010591D990D112CD
:107440000D2D08B94C910591D990D1120D2D08B987
:10745000429F0591D990D1120D2D08B9040C151C2D
:107460000591D990D1120D2D08B9080E191E05915C
:10747000D990D1120D2D08B9A395AF710591D9906E
:10748000D1120D2D08B9A32BF0010591D990D1127D
:107490000D2D08B94C910591D990D1120D2D08B937
:1074A000429F0591D990D1120D2D08B9040C151CDD
:1074B0000591D990D1120D2D08B9080E191E05910C
:1074C000D990D1120D2D08B9A395AF710591D9901E
:1074D000D1120D2D08B9A32BF0010591D990D1122D
:1074E0000D2D08B94C910591D990D1120D2D08B9E7
:1074F000429F0591D990D1120D2D08B9040C151C8D
:107500000591D990D1120D2D08B9080E191E0591BB
:10751000D990D1120D2D08B9A395AF710591D990CD
:10752000D1120D2D08B9A32BF0010591D990D112DC
:107530000D2D08B94C910591D990D1120D2D08B996
:10754000429F0591D990D1120D2D08B9040C151C3C
:107550000591D990D1120D2D08B9080E191E05916B
:10756000D990D1120D2D08B9A395AF710591D9907D
:10757000D1120D2D08B9A32BF0010591D990D1128C
:107580000D2D08B94C910591D990D1120D2D08B946
:10759000429F0591D990D1120D2D08B9040C151CEC
:1075A0000591D990D1120D2D08B9080E191E05911B
:1075B000D990D1120D2D08B9A395AF710591D9902D
:1075C000D1120D2D08B9A32BF0010591D990D1123C
:1075D0000D2D08B94C910591D990D1120D2D08B9F6
:1075E000429F0591D990D1120D2D08B9040C151C9C
:1075F0000591D990D1120D2D08B9080E191E0591CB
:10760000D990D1120D2D08B9A395AF710591D990DC
:10761000D1120D2D08B9A32BF0010591D990D112EB
:107620000D2D08B94C910591D990D1120D2D08B9A5
:10763000429F0591D990D1120D2D08B9040C151C4B
:107640000591D990D1120D2D08B9080E191E05917A
:10765000D990D1120D2D08B9A395AF710591D9908C
:10766000D1120D2D08B9A32BF0010591D990D1129B
:107670000D2D08B94C910591D990D1120D2D08B955
:10768000429F0591D990D1120D2D08B9040C151CFB
:107690000591D990D1120D2D08B9080E191E05912A
:1076A000D990D1120D2D08B9A395AF710591D9903C
:1076B000D1120D2D08B9A32BF0010591D990D1124B
:1076C0000D2D08B94C910591D990D1120D2D08B905
:1076D000429F0591D990D1120D2D08B9040C151CAB
:1076E0000591D990D1120D2D08B9080E191E0591DA
:1076F000D990D1120D2D08B9A395AF710591D990EC
:10770000D1120D2D08B9A32BF0010591D990D112FA
:107710000D2D08B94C910591D990D1120D2D08B9B4
:10772000429F0591D990D1120D2D08B9040C151C5A
:107730000591D990D1120D2D08B9080E191E059189
:10774000D990D1120D2D08B9A395AF710591D9909B
:10775000D1120D2D08B9A32BF0010591D990D112AA
:107760000D2D08B94C910591D990D1120D2D08B964
:10777000429F0591D990D1120D2D08B9040C151C0A
:107780000591D990D1120D2D08B9080E191E059139
:10779000D990D1120D2D08B9A395AF710591D9904B
:1077A000D1120D2D08B9A32BF0010591D990D1125A
:1077B0000D2D08B94C910591D990D1120D2D08B914
:1077C000429F0591D990D1120D2D08B9040C151CBA
:1077D0000591D990D1120D2D08B9080E191E0591E9
:1077E000D990D1120D2D08B9A395AF710591D990FB
:1077F000D1120D2D08B9A32BF0010591D990D1120A
:107800000D2D08B94C910591D990D1120D2D08B9C3
:10781000429F0591D990D1120D2D08B9040C151C69
:107820000591D990D1120D2D08B9080E191E059198
:10783000D990D1120D2D08B9A395AF710591D990AA
:10784000D1120D2D08B9A32BF0010591D990D112B9
:107850000D2D08B94C910591D990D1120D2D08B973
:10786000429F0591D990D1120D2D08B9040C151C19
:107870000591D990D1120D2D08B9080E191E059148
:10788000D990D1120D2D08B9A395AF710591D9905A
:10789000D1120D2D08B9A32BF0010591D990D11269
:1078A0000D2D08B94C912F91000000000027D30145
:1078B000E10108B90895F00132964C91429F00C051
:1078C00000C000C00591D990D1120D2D08B9040C4B
:1078D000151C0591D990D1120D2D08B9080E191E4D
:1078E0000591D990D1120D2D08B9A395AF710591CD
:1078F000D990D1120D2D08B9A32BF0010591D99083
:10790000D1120D2D08B94C910591D990D1120D2DA0
:1079100008B9429F0591D990D1120D2D08B9040CD8
:10792000151C0591D990D1120D2D08B9080E191EFC
:107930000591D990D1120D2D08B9A395AF7105917C
:10794000D990D1120D2D08B9A32BF0010591D99032
:10795000D1120D2D08B94C910591D990D1120D2D50
:1079600008B9429F0591D990D1120D2D08B9040C88
:10797000151C0591D990D1120D2D08B9080E191EAC
:107980000591D990D1120D2D08B9A395AF7105912C
:10799000D990D1120D2D08B9A32BF0010591D990E2
:1079A000D1120D2D08B94C910591D990D1120D2D00
:1079B00008B9429F0591D990D1120D2D08B9040C38
:1079C000151C0591D990D1120D2D08B9080E191E5C
:1079D0000591D990D1120D2D08B9A395AF710591DC
:1079E000D990D1120D2D08B9A32BF0010591D99092
:1079F000D1120D2D08B94C910591D990D1120D2DB0
:107A000008B9429F0591D990D1120D2D08B9040CE7
:107A1000151C0591D990D1120D2D08B9080E191E0B
:107A20000591D990D1120D2D08B9A395AF7105918B
:107A3000D990D1120D2D08B9A32BF0010591D99041
:107A4000D1120D2D08B94C910591D990D1120D2D5F
:107A500008B9429F0591D990D1120D2D08B9040C97
:107A6000151C0591D990D1120D2D08B9080E191EBB
:107A70000591D990D1120D2D08B9A395AF7105913B
:107A8000D990D1120D2D08B9A32BF0010591D990F1
:107A9000D1120D2D08B94C910591D990D1120D2D0F
:107AA00008B9429F0591D990D1120D2D08B9040C47
:107AB000151C0591D990D1120D2D08B9080E191E6B
:107AC0000591D990D1120D2D08B9A395AF710591EB
:107AD000D990D1120D2D08B9A32BF0010591D990A1
:107AE000D1120D2D08B94C910591D990D1120D2DBF
:107AF00008B9429F0591D990D1120D2D08B9040CF7
:107B0000151C0591D990D1120D2D08B9080E191E1A
:107B10000591D990D1120D2D08B9A395AF7105919A
:107B2000D990D1120D2D08B9A32BF0010591D99050
:107B3000D1120D2D08B94C910591D990D1120D2D6E
:107B400008B9429F0591D990D1120D2D08B9040CA6
:107B5000151C0591D990D1120D2D08B9080E191ECA
:107B60000591D990D1120D2D08B9A395AF7105914A
:107B7000D990D1120D2D08B9A32BF0010591D99000
:107B8000D1120D2D08B94C910591D990D1120D2D1E
:107B900008B9429F0591D990D1120D2D08B9040C56
:107BA000151C0591D990D1120D2D08B9080E191E7A
:107BB0000591D990D1120D2D08B9A395AF710591FA
:107BC000D990D1120D2D08B9A32BF0010591D990B0
:107BD000D1120D2D08B94C910591D990D1120D2DCE
:107BE00008B9429F0591D990D1120D2D08B9040C06
:107BF000151C0591D990D1120D2D08B9080E191E2A
:107C00000591D990D1120D2D08B9A395AF710591A9
:107C1000D990D1120D2D08B9A32BF0010591D9905F
:107C2000D1120D2D08B94C910591D990D1120D2D7D
:107C300008B9429F0591D990D1120D2D08B9040CB5
:107C4000151C0591D990D1120D2D08B9080E191ED9
:107C50000591D990D1120D2D08B9A395AF71059159
:107C6000D990D1120D2D08B9A32BF0010591D9900F
:107C7000D1120D2D08B94C910591D990D1120D2D2D
:107C800008B9429F0591D990D1120D2D08B9040C65
:107C9000151C0591D990D1120D2D08B9080E191E89
:107CA0000591D990D1120D2D08B9A395AF71059109
:107CB000D990D1120D2D08B9A32BF0010591D990BF
:107CC000D1120D2D08B94C910591D990D1120D2DDD
:107CD00008B9429F0591D990D1120D2D08B9040C15
:107CE000151C0591D990D1120D2D08B9080E191E39
:107CF0000591D990D1120D2D08B9A395AF710591B9
:107D0000D990D1120D2D08B9A32BF0010591D9906E
:107D1000D1120D2D08B94C910591D990D1120D2D8C
:107D200008B9429F0591D990D1120D2D08B9040CC4
:107D3000151C0591D990D1120D2D08B9080E191EE8
:107D40000591D990D1120D2D08B9A395AF71059168
:107D5000D990D1120D2D08B9A32BF0010591D9901E
:107D6000D1120D2D08B94C910591D990D1120D2D3C
:107D700008B9429F0591D990D1120D2D08B9040C74
:107D8000151C0591D990D1120D2D08B9080E191E98
:107D90000591D990D1120D2D08B9A395AF71059118
:107DA000D990D1120D2D08B9A32BF0010591D990CE
:107DB000D1120D2D08B94C910591D990D1120D2DEC
:107DC00008B9429F0591D990D1120D2D08B9040C24
:107DD000151C0591D990D1120D2D08B9080E191E48
:107DE0000591D990D1120D2D08B9A395AF710591C8
:107DF000D990D1120D2D08B9A32BF0010591D9907E
:107E0000D1120D2D08B94C910591D990D1120D2D9B
:107E100008B9429F0591D990D1120D2D08B9040CD3
:107E2000151C0591D990D1120D2D08B9080E191EF7
:107E30000591D990D1120D2D08B9A395AF71059177
:107E4000D990D1120D2D08B9A32BF0010591D9902D
:107E5000D1120D2D08B94C910591D990D1120D2D4B
:107E600008B9429F0591D990D1120D2D08B9040C83
:107E7000151C0591D990D1120D2D08B9080E191EA7
:107E80000591D990D1120D2D08B9A395AF71059127
:107E9000D990D1120D2D08B9A32BF0010591D990DD
:107EA000D1120D2D08B94C910591D990D1120D2DFB
:107EB00008B9429F0591D990D1120D2D08B9040C33
:107EC000151C0591D990D1120D2D08B9080E191E57
:107ED0000591D990D1120D2D08B9A395AF710591D7
:107EE000D990D1120D2D08B9A32BF0010591D9908D
:107EF000D1120D2D08B94C910591D990D1120D2DAB
:107F000008B9429F0591D990D1120D2D08B9040CE2
:107F1000151C0591D990D1120D2D08B9080E191E06
:107F20000591D990D1120D2D08B9A395AF71059186
:107F3000D990D1120D2D08B9A32BF0010591D9903C
:107F4000D1120D2D08B94C910591D990D1120D2D5A
:107F500008B9429F0591D990D1120D2D08B9040C92
:107F6000151C0591D990D1120D2D08B9080E191EB6
:107F70000591D990D1120D2D08B9A395AF71059136
:107F8000D990D1120D2D08B9A32BF0010591D990EC
:107F9000D1120D2D08B94C910591D990D1120D2D0A
:107FA00008B9429F2F91000000000027D301E10192
:107FB00008B90895F00133964C91429F040C151CAA
:107FC00000C000C00591D990D1120D2D08B9080E3E
:107FD000191E0591D990D1120D2D08B9A395AF7135
:107FE0000591D990D1120D2D08B9A32BF00105915F
:107FF000D990D1120D2D08B94C910591D990D1127B
:108000000D2D08B9429F0591D990D1120D2D08B9B7
:10801000040C151C0591D990D1120D2D08B9080E2C
:10802000191E0591D990D1120D2D08B9A395AF71E4
:108030000591D990D1120D2D08B9A32BF00105910E
:10804000D990D1120D2D08B94C910591D990D1122A
:108050000D2D08B9429F0591D990D1120D2D08B967
:10806000040C151C0591D990D1120D2D08B9080EDC
:10807000191E0591D990D1120D2D08B9A395AF7194
:108080000591D990D1120D2D08B9A32BF0010591BE
:10809000D990D1120D2D08B94C910591D990D112DA
:1080A0000D2D08B9429F0591D990D1120D2D08B917
:1080B000040C151C0591D990D1120D2D08B9080E8C
:1080C000191E0591D990D1120D2D08B9A395AF7144
:1080D0000591D990D1120D2D08B9A32BF00105916E
:1080E000D990D1120D2D08B94C910591D990D1128A
:1080F0000D2D08B9429F0591D990D1120D2D08B9C7
:10810000040C151C0591D990D1120D2D08B9080E3B
:10811000191E0591D990D1120D2D08B9A395AF71F3
:108120000591D990D1120D2D08B9A32BF00105911D
:10813000D990D1120D2D08B94C910591D990D11239
:108140000D2D08B9429F0591D990D1120D2D08B976
:10815000040C151C0591D990D1120D2D08B9080EEB
:10816000191E0591D990D1120D2D08B9A395AF71A3
:108170000591D990D1120D2D08B9A32BF0010591CD
:10818000D990D1120D2D08B94C910591D990D112E9
:108190000D2D08B9429F0591D990D1120D2D08B926
:1081A000040C151C0591D990D1120D2D08B9080E9B
:1081B000191E0591D990D1120D2D08B9A395AF7153
:1081C0000591D990D1120D2D08B9A32BF00105917D
:1081D000D990D1120D2D08B94C910591D990D11299
:1081E0000D2D08B9429F0591D990D1120D2D08B9D6
:1081F000040C151C0591D990D1120D2D08B9080E4B
:10820000191E0591D990D1120D2D08B9A395AF7102
:108210000591D990D1120D2D08B9A32BF00105912C
:10822000D990D1120D2D08B94C910591D990D11248
:108230000D2D08B9429F0591D990D1120D2D08B985
:10824000040C151C0591D990D1120D2D08B9080EFA
:10825000191E0591D990D1120D2D08B9A395AF71B2
:108260000591D990D1120D2D08B9A32BF0010591DC
:10827000D990D1120D2D08B94C910591D990D112F8
:108280000D2D08B9429F0591D990D1120D2D08B935
:10829000040C151C0591D990D1120D2D08B9080EAA
:1082A000191E0591D990D1120D2D08B9A395AF7162
:1082B0000591D990D1120D2D08B9A32BF00105918C
:1082C000D990D1120D2D08B94C910591D990D112A8
:1082D0000D2D08B9429F0591D990D1120D2D08B9E5
:1082E000040C151C0591D990D1120D2D08B9080E5A
:1082F000191E0591D990D1120D2D08B9A395AF7112
:108300000591D990D1120D2D08B9A32BF00105913B
:10831000D990D1120D2D08B94C910591D990D11257
:108320000D2D08B9429F0591D990D1120D2D08B994
:10833000040C151C0591D990D1120D2D08B9080E09
:10834000191E0591D990D1120D2D08B9A395AF71C1
:108350000591D990D1120D2D08B9A32BF0010591EB
:10836000D990D1120D2D08B94C910591D990D11207
:108370000D2D08B9429F0591D990D1120D2D08B944
:10838000040C151C0591D990D1120D2D08B9080EB9
:10839000191E0591D990D1120D2D08B9A395AF7171
:1083A0000591D990D1120D2D08B9A32BF00105919B
:1083B000D990D1120D2D08B94C910591D990D112B7
:1083C0000D2D08B9429F0591D990D1120D2D08B9F4
:1083D000040C151C0591D990D1120D2D08B9080E69
:1083E000191E0591D990D1120D2D08B9A395AF7121
:1083F0000591D990D1120D2D08B9A32BF00105914B
:10840000D990D1120D2D08B94C910591D990D11266
:108410000D2D08B9429F0591D990D1120D2D08B9A3
:10842000040C151C0591D990D1120D2D08B9080E18
:10843000191E0591D990D1120D2D08B9A395AF71D0
:108440000591D990D1120D2D08B9A32BF0010591FA
:10845000D990D1120D2D08B94C910591D990D11216
:108460000D2D08B9429F0591D990D1120D2D08B953
:10847000040C151C0591D990D1120D2D08B9080EC8
:10848000191E0591D990D1120D2D08B9A395AF7180
:108490000591D990D1120D2D08B9A32BF0010591AA
:1084A000D990D1120D2D08B94C910591D990D112C6
:1084B0000D2D08B9429F0591D990D1120D2D08B903
:1084C000040C151C0591D990D1120D2D08B9080E78
:1084D000191E0591D990D1120D2D08B9A395AF7130
:1084E0000591D990D1120D2D08B9A32BF00105915A
:1084F000D990D1120D2D08B94C910591D990D11276
:108500000D2D08B9429F0591D990D1120D2D08B9B2
:10851000040C151C0591D990D1120D2D08B9080E27
:10852000191E0591D990D1120D2D08B9A395AF71DF
:108530000591D990D1120D2D08B9A32BF001059109
:10854000D990D1120D2D08B94C910591D990D11225
:108550000D2D08B9429F0591D990D1120D2D08B962
:10856000040C151C0591D990D1120D2D08B9080ED7
:10857000191E0591D990D1120D2D08B9A395AF718F
:108580000591D990D1120D2D08B9A32BF0010591B9
:10859000D990D1120D2D08B94C910591D990D112D5
:1085A0000D2D08B9429F0591D990D1120D2D08B912
:1085B000040C151C0591D990D1120D2D08B9080E87
:1085C000191E0591D990D1120D2D08B9A395AF713F
:1085D0000591D990D1120D2D08B9A32BF001059169
:1085E000D990D1120D2D08B94C910591D990D11285
:1085F0000D2D08B9429F0591D990D1120D2D08B9C2
:10860000040C151C0591D990D1120D2D08B9080E36
:10861000191E0591D990D1120D2D08B9A395AF71EE
:108620000591D990D1120D2D08B9A32BF001059118
:10863000D990D1120D2D08B94C910591D990D11234
:108640000D2D08B9429F0591D990D1120D2D08B971
:10865000040C151C0591D990D1120D2D08B9080EE6
:10866000191E0591D990D1120D2D08B9A395AF719E
:108670000591D990D1120D2D08B9A32BF0010591C8
:10868000D990D1120D2D08B94C910591D990D112E4
:108690000D2D08B9429F0591D990D1120D2D08B921
:1086A000040C151C2F91000000000027D301E101EC
:1086B00008B90895F00134964C91429F040C151CA2
:1086C000080E191E00C00591D990D1120D2D08B9C0
:1086D000A395AF710591D990D1120D2D08B9A32B97
:1086E000F0010591D990D1120D2D08B94C91059149
:1086F000D990D1120D2D08B9429F0591D990D11270
:108700000D2D08B9040C151C0591D990D1120D2D11
:1087100008B9080E191E0591D990D1120D2D08B96E
:10872000A395AF710591D990D1120D2D08B9A32B46
:10873000F0010591D990D1120D2D08B94C910591F8
:10874000D990D1120D2D08B9429F0591D990D1121F
:108750000D2D08B9040C151C0591D990D1120D2DC1
:1087600008B9080E191E0591D990D1120D2D08B91E
:10877000A395AF710591D990D1120D2D08B9A32BF6
:10878000F0010591D990D1120D2D08B94C910591A8
:10879000D990D1120D2D08B9429F0591D990D112CF
:1087A0000D2D08B9040C151C0591D990D1120D2D71
:1087B00008B9080E191E0591D990D1120D2D08B9CE
:1087C000A395AF710591D990D1120D2D08B9A32BA6
:1087D000F0010591D990D1120D2D08B94C91059158
:1087E000D990D1120D2D08B9429F0591D990D1127F
:1087F0000D2D08B9040C151C0591D990D1120D2D21
:1088000008B9080E191E0591D990D1120D2D08B97D
:10881000A395AF710591D990D1120D2D08B9A32B55
:10882000F0010591D990D1120D2D08B94C91059107
:10883000D990D1120D2D08B9429F0591D990D1122E
:108840000D2D08B9040C151C0591D990D1120D2DD0
:1088500008B9080E191E0591D990D1120D2D08B92D
:10886000A395AF710591D990D1120D2D08B9A32B05
:10887000F0010591D990D1120D2D08B94C910591B7
:10888000D990D1120D2D08B9429F0591D990D112DE
:108890000D2D08B9040C151C0591D990D1120D2D80
:1088A00008B9080E191E0591D990D1120D2D08B9DD
:1088B000A395AF710591D990D1120D2D08B9A32BB5
:1088C000F0010591D990D1120D2D08B94C91059167
:1088D000D990D1120D2D08B9429F0591D990D1128E
:1088E0000D2D08B9040C151C0591D990D1120D2D30
:1088F00008B9080E191E0591D990D1120D2D08B98D
:10890000A395AF710591D990D1120D2D08B9A32B64
:10891000F0010591D990D1120D2D08B94C91059116
:10892000D990D1120D2D08B9429F0591D990D1123D
:108930000D2D08B9040C151C0591D990D1120D2DDF
:1089400008B9080E191E0591D990D1120D2D08B93C
:10895000A395AF710591D990D1120D2D08B9A32B14
:10896000F0010591D990D1120D2D08B94C910591C6
:10897000D990D1120D2D08B9429F0591D990D112ED
:108980000D2D08B9040C151C0591D990D1120D2D8F
:1089900008B9080E191E0591D990D1120D2D08B9EC
:1089A000A395AF710591D990D1120D2D08B9A32BC4
:1089B000F0010591D990D1120D2D08B94C91059176
:1089C000D990D1120D2D08B9429F0591D990D1129D
:1089D0000D2D08B9040C151C0591D990D1120D2D3F
:1089E00008B9080E191E0591D990D1120D2D08B99C
:1089F000A395AF710591D990D1120D2D08B9A32B74
:108A0000F0010591D990D1120D2D08B94C91059125
:108A1000D990D1120D2D08B9429F0591D990D1124C
:108A20000D2D08B9040C151C0591D990D1120D2DEE
:108A300008B9080E191E0591D990D1120D2D08B94B
:108A4000A395AF710591D990D1120D2D08B9A32B23
:108A5000F0010591D990D1120D2D08B94C910591D5
:108A6000D990D1120D2D08B9429F0591D990D112FC
:108A70000D2D08B9040C151C0591D990D1120D2D9E
:108A800008B9080E191E0591D990D1120D2D08B9FB
:108A9000A395AF710591D990D1120D2D08B9A32BD3
:108AA000F0010591D990D1120D2D08B94C91059185
:108AB000D990D1120D2D08B9429F0591D990D112AC
:108AC0000D2D08B9040C151C0591D990D1120D2D4E
:108AD00008B9080E191E0591D990D1120D2D08B9AB
:108AE000A395AF710591D990D1120D2D08B9A32B83
:108AF000F0010591D990D1120D2D08B94C91059135
:108B0000D990D1120D2D08B9429F0591D990D1125B
:108B10000D2D08B9040C151C0591D990D1120D2DFD
:108B200008B9080E191E0591D990D1120D2D08B95A
:108B3000A395AF710591D990D1120D2D08B9A32B32
:108B4000F0010591D990D1120D2D08B94C910591E4
:108B5000D990D1120D2D08B9429F0591D990D1120B
:108B60000D2D08B9040C151C0591D990D1120D2DAD
:108B700008B9080E191E0591D990D1120D2D08B90A
:108B8000A395AF710591D990D1120D2D08B9A32BE2
:108B9000F0010591D990D1120D2D08B94C91059194
:108BA000D990D1120D2D08B9429F0591D990D112BB
:108BB0000D2D08B9040C151C0591D990D1120D2D5D
:108BC00008B9080E191E0591D990D1120D2D08B9BA
:108BD000A395AF710591D990D1120D2D08B9A32B92
:108BE000F0010591D990D1120D2D08B94C91059144
:108BF000D990D1120D2D08B9429F0591D990D1126B
:108C00000D2D08B9040C151C0591D990D1120D2D0C
:108C100008B9080E191E0591D990D1120D2D08B969
:108C2000A395AF710591D990D1120D2D08B9A32B41
:108C3000F0010591D990D1120D2D08B94C910591F3
:108C4000D990D1120D2D08B9429F0591D990D1121A
:108C50000D2D08B9040C151C0591D990D1120D2DBC
:108C600008B9080E191E0591D990D1120D2D08B919
:108C7000A395AF710591D990D1120D2D08B9A32BF1
:108C8000F0010591D990D1120D2D08B94C910591A3
:108C9000D990D1120D2D08B9429F0591D990D112CA
:108CA0000D2D08B9040C151C0591D990D1120D2D6C
:108CB00008B9080E191E0591D990D1120D2D08B9C9
:108CC000A395AF710591D990D1120D2D08B9A32BA1
:108CD000F0010591D990D1120D2D08B94C91059153
:108CE000D990D1120D2D08B9429F0591D990D1127A
:108CF0000D2D08B9040C151C0591D990D1120D2D1C
:108D000008B9080E191E0591D990D1120D2D08B978
:108D1000A395AF710591D990D1120D2D08B9A32B50
:108D2000F0010591D990D1120D2D08B94C91059102
:108D3000D990D1120D2D08B9429F0591D990D11229
:108D40000D2D08B9040C151C0591D990D1120D2DCB
:108D500008B9080E191E0591D990D1120D2D08B928
:108D6000A395AF710591D990D1120D2D08B9A32B00
:108D7000F0010591D990D1120D2D08B94C910591B2
:108D8000D990D1120D2D08B9429F0591D990D112D9
:108D90000D2D08B9040C151C0591D990D1120D2D7B
:108DA00008B9080E191E2F91000000000027D301FA
:108DB000E10108B90895F00135964C91429F040CE9
:108DC000151C080E191EA395AF710591D990D112EB
:108DD0000D2D08B9A32BF0010591D990D1120D2DBD
:108DE00008B94C910591D990D1120D2D08B9429F27
:108DF0000591D990D1120D2D08B9040C151C0591BF
:108E0000D990D1120D2D08B9080E191E0591D990CF
:108E1000D1120D2D08B9A395AF710591D990D1123A
:108E20000D2D08B9A32BF0010591D990D1120D2D6C
:108E300008B94C910591D990D1120D2D08B9429FD6
:108E40000591D990D1120D2D08B9040C151C05916E
:108E5000D990D1120D2D08B9080E191E0591D9907F
:108E6000D1120D2D08B9A395AF710591D990D112EA
:108E70000D2D08B9A32BF0010591D990D1120D2D1C
:108E800008B94C910591D990D1120D2D08B9429F86
:108E90000591D990D1120D2D08B9040C151C05911E
:108EA000D990D1120D2D08B9080E191E0591D9902F
:108EB000D1120D2D08B9A395AF710591D990D1129A
:108EC0000D2D08B9A32BF0010591D990D1120D2DCC
:108ED00008B94C910591D990D1120D2D08B9429F36
:108EE0000591D990D1120D2D08B9040C151C0591CE
:108EF000D990D1120D2D08B9080E191E0591D990DF
:108F0000D1120D2D08B9A395AF710591D990D11249
:108F10000D2D08B9A32BF0010591D990D1120D2D7B
:108F200008B94C910591D990D1120D2D08B9429FE5
:108F30000591D990D1120D2D08B9040C151C05917D
:108F4000D990D1120D2D08B9080E191E0591D9908E
:108F5000D1120D2D08B9A395AF710591D990D112F9
:108F60000D2D08B9A32BF0010591D990D1120D2D2B
:108F700008B94C910591D990D1120D2D08B9429F95
:108F80000591D990D1120D2D08B9040C151C05912D
:108F9000D990D1120D2D08B9080E191E0591D9903E
:108FA000D1120D2D08B9A395AF710591D990D112A9
:108FB0000D2D08B9A32BF0010591D990D1120D2DDB
:108FC00008B94C910591D990D1120D2D08B9429F45
:108FD0000591D990D1120D2D08B9040C151C0591DD
:108FE000D990D1120D2D08B9080E191E0591D990EE
:108FF000D1120D2D08B9A395AF710591D990D11259
:109000000D2D08B9A32BF0010591D990D1120D2D8A
:1090100008B94C910591D990D1120D2D08B9429FF4
:109020000591D990D1120D2D08B9040C151C05918C
:10903000D990D1120D2D08B9080E191E0591D9909D
:10904000D1120D2D08B9A395AF710591D990D11208
:109050000D2D08B9A32BF0010591D990D1120D2D3A
:1090600008B94C910591D990D1120D2D08B9429FA4
:109070000591D990D1120D2D08B9040C151C05913C
:10908000D990D1120D2D08B9080E191E0591D9904D
:10909000D1120D2D08B9A395AF710591D990D112B8
:1090A0000D2D08B9A32BF0010591D990D1120D2DEA
:1090B00008B94C910591D990D1120D2D08B9429F54
:1090C0000591D990D1120D2D08B9040C151C0591EC
:1090D000D990D1120D2D08B9080E191E0591D990FD
:1090E000D1120D2D08B9A395AF710591D990D11268
:1090F0000D2D08B9A32BF0010591D990D1120D2D9A
:1091000008B94C910591D990D1120D2D08B9429F03
:109110000591D990D1120D2D08B9040C151C05919B
:10912000D990D1120D2D08B9080E191E0591D990AC
:10913000D1120D2D08B9A395AF710591D990D11217
:109140000D2D08B9A32BF0010591D990D1120D2D49
:1091500008B94C910591D990D1120D2D08B9429FB3
:109160000591D990D1120D2D08B9040C151C05914B
:10917000D990D1120D2D08B9080E191E0591D9905C
:10918000D1120D2D08B9A395AF710591D990D112C7
:109190000D2D08B9A32BF0010591D990D1120D2DF9
:1091A00008B94C910591D990D1120D2D08B9429F63
:1091B0000591D990D1120D2D08B9040C151C0591FB
:1091C000D990D1120D2D08B9080E191E0591D9900C
:1091D000D1120D2D08B9A395AF710591D990D11277
:1091E0000D2D08B9A32BF0010591D990D1120D2DA9
:1091F00008B94C910591D990D1120D2D08B9429F13
:109200000591D990D1120D2D08B9040C151C0591AA
:10921000D990D1120D2D08B9080E191E0591D990BB
:10922000D1120D2D08B9A395AF710591D990D11226
:109230000D2D08B9A32BF0010591D990D1120D2D58
:1092400008B94C910591D990D1120D2D08B9429FC2
:109250000591D990D1120D2D08B9040C151C05915A
:10926000D990D1120D2D08B9080E191E0591D9906B
:10927000D1120D2D08B9A395AF710591D990D112D6
:109280000D2D08B9A32BF0010591D990D1120D2D08
:1092900008B94C910591D990D1120D2D08B9429F72
:1092A0000591D990D1120D2D08B9040C151C05910A
:1092B000D990D1120D2D08B9080E191E0591D9901B
:1092C000D1120D2D08B9A395AF710591D990D11286
:1092D0000D2D08B9A32BF0010591D990D1120D2DB8
:1092E00008B94C910591D990D1120D2D08B9429F22
:1092F0000591D990D1120D2D08B9040C151C0591BA
:10930000D990D1120D2D08B9080E191E0591D990CA
:10931000D1120D2D08B9A395AF710591D990D11235
:109320000D2D08B9A32BF0010591D990D1120D2D67
:1093300008B94C910591D990D1120D2D08B9429FD1
:109340000591D990D1120D2D08B9040C151C059169
:10935000D990D1120D2D08B9080E191E0591D9907A
:10936000D1120D2D08B9A395AF710591D990D112E5
:109370000D2D08B9A32BF0010591D990D1120D2D17
:1093800008B94C910591D990D1120D2D08B9429F81
:109390000591D990D1120D2D08B9040C151C059119
:1093A000D990D1120D2D08B9080E191E0591D9902A
:1093B000D1120D2D08B9A395AF710591D990D11295
:1093C0000D2D08B9A32BF0010591D990D1120D2DC7
:1093D00008B94C910591D990D1120D2D08B9429F31
:1093E0000591D990D1120D2D08B9040C151C0591C9
:1093F000D990D1120D2D08B9080E191E0591D990DA
:10940000D1120D2D08B9A395AF710591D990D11244
:109410000D2D08B9A32BF0010591D990D1120D2D76
:1094200008B94C910591D990D1120D2D08B9429FE0
:109430000591D990D1120D2D08B9040C151C059178
:10944000D990D1120D2D08B9080E191E0591D99089
:10945000D1120D2D08B9A395AF710591D990D112F4
:109460000D2D08B9A32BF0010591D990D1120D2D26
:1094700008B94C910591D990D1120D2D08B9429F90
:109480000591D990D1120D2D08B9040C151C059128
:10949000D990D1120D2D08B9080E191E0591D99039
:1094A000D1120D2D08B9A395AF712F9100000000C6
:1094B0000027D301E10108B90895CC03CC03CC0304
:1094C000CC03CC03CC03CC03CC03CC03CC03CC0324
:1094D000CC03CC03CC03CC03CC03CC03CC03CC0314
:1094E000CC03CC03CC03CC03CC03CC03CC03CC0304
:1094F000CC03CC03CC03CC03CC03CC03CC03CC03F4
:10950000CC03CC03CC03CC03CC03CC03CC03CC03E3
:10951000CC03CC03CC03CC03CC03CC03CC032898E2
:109520000E94812BE7E1EA95F1F7289A05D1E0E066
:10953000F6E0E8D0E0FF43D0E0FF02C00E94472AF7
:109540000895129A0C94A44A0C94A64A129844279F
:109550005527662777278CE00C94AE4A0C94B04AC6
:109560000C94B24A0C94B44A0C94B64A0C94B84A7F
:10957000440F551F00994160660F771F0199616084
:10958000139A0C94C34A0C94C54A13980C94C84A75
:109590000C94CA4A0C94CC4A0C94CE4A8A9541F752
:1095A00040955095609570955F707F7040930B0C5F
:1095B00050930C0C60930D0C70930E0C0895EF9368
:1095C000E091010CE43EE0F5E431D0F12F923F92BE
:1095D0004F925F926F927F928F929F92AF92BF92C3
:1095E000CF92DF92EF92FF920F931F932F933F93AF
:1095F0004F935F936F937F938F939F93AF93BF939B
:10960000CF93DF930E940734DF91CF91BF91AF9149
:109610009F918F917F916F915F914F913F912F918A
:109620001F910F91FF90EF90DF90CF90BF90AF9080
:109630009F908F907F906F905F904F903F902F9072
:10964000EF910895FF93EF93EFB7EF93E0918400CC
:10965000EE50E13000F0E23000F0E33000F0E430B2
:1096600000F0E53000F0E63000F0E73000F0E830E0
:1096700000F0E93000F005D0EF91EFBFEF91FF91DE
:1096800018950F921F92EAEFF7E60090000C000C7D
:109690001124E00DF11D05901490F00109951F9023
:1096A0000F90089528980E94812BE5E1EA95F1F743
:1096B000E091010CEA95E093010C289A000000006B
:1096C000089528980E94AA2B289A0000E1E0F6E06D
:1096D00019D02BD0089528980E94AA2BE0EB000007
:1096E000EA95E9F700000000289AF6E0E2E00AD0E7
:1096F000089528980E94AA2B289A0000E3E0FCEF26
:1097000001D008950090010C0A9410905F0011FCA4
:109710000F2E0092010C0090000C11FC0E2E0092F6
:10972000000CE0E011FCE1E00895E3E0E093890043
:10973000EDE8E09388000895E7E0E0938900EBE12D
:10974000E09388000895E0E6F4E0A0E6B3E0662741
:109750006D933197E9F7112408959927772720E22F
:10976000629F080E191EA0E6B3E0A00DB11D4C9338
:10977000112408950895992720E2629F080E191E6A
:10978000A0E6B3E0A00DB11D50910A0C450F4C931B
:109790001124089580930A0C0895F8944427409367
:1097A0008100409345004FEF47B944B940E84AB9BA
:1097B0004CE041B900E00093000C06E00093010C7E
:1097C000409385004093840043E0409389004DE836
:1097D0004093880049E04093810042E040936F004D
:1097E00042E44093440040E04093470041E00000E1
:1097F0004093450043E84093B00040E04093B300FD
:1098000041E04093B10041E145B97894112440E929
:10981000A3ECB7E00EEF0D934A95E9F740E04093D3
:10982000C00708958093080C9093090C08958093C5
:10983000040C9093050C08958093060C9093070CEC
:1098400008958091020C089511241092020C08953D
:10985000882329F480910B0C90910C0C0895809131
:109860000D0C90910E0C089580E891E080936100BA
:1098700090936100089580E890E080936100909358
:10988000610008958093FB0B9093FC0B08958093E7
:10989000C0070895A0E0B0E0E0E5FCE40C94424D80
:1098A000EC01A880B980CA80DB80A114B104C10496
:1098B000D10441F484E2A82E89EDB82E8BE5C82EA0
:1098C00087E0D82EC601B5012DE133EF41E050E02D
:1098D0000E941F4D27EA31E440E050E00E94004D15
:1098E0007B018C01C601B5012DE133EF41E050E071
:1098F0000E941F4DCA01B9012CEE34EF4FEF5FEF0C
:109900000E94004D6E0D7F1D801F911F97FF04C0A8
:109910006150704080409048688379838A839B833C
:109920009B013F77C901CDB7DEB7EAE00C945E4DED
:109930000E944A4C089589E191E00E944A4C0895A2
:10994000A0E0B0E08093190190931A01A0931B014D
:10995000B0931C010895991B79E004C0991F9617D4
:1099600008F0961B881F7A95C9F78095089597FB94
:10997000092E07260AD077FD04D02ED006D000206D
:109980001AF4709561957F4F0895F6F7909581953B
:109990009F4F0895A1E21A2EAA1BBB1BFD010DC00B
:1099A000AA1FBB1FEE1FFF1FA217B307E407F5078F
:1099B00020F0A21BB30BE40BF50B661F771F881F6B
:1099C000991F1A9469F760957095809590959B0101
:1099D000AC01BD01CF010895AA1BBB1B51E107C01B
:1099E000AA1FBB1FA617B70710F0A61BB70B881F2F
:1099F000991F5A95A9F780959095BC01CD010895BE
:109A0000629FD001739FF001829FE00DF11D649F62
:109A1000E00DF11D929FF00D839FF00D749FF00DEE
:109A2000659FF00D9927729FB00DE11DF91F639F8F
:109A3000B00DE11DF91FBD01CF011124089597FB61
:109A4000092E05260ED057FD04D0A4DF0AD0001C35
:109A500038F450954095309521953F4F4F4F5F4FCB
:109A60000895F6F790958095709561957F4F8F4F8B
:109A70009F4F08952F923F924F925F926F927F92E5
:109A80008F929F92AF92BF92CF92DF92EF92FF920E
:109A90000F931F93CF93DF93CDB7DEB7CA1BDB0BBA
:109AA0000FB6F894DEBF0FBECDBF09942A8839885F
:109AB00048885F846E847D848C849B84AA84B98466
:109AC000C884DF80EE80FD800C811B81AA81B98172
:109AD000CE0FD11D0FB6F894DEBF0FBECDBFED0186
:069AE0000895F894FFCF89
:109AE6003CC30361256F257F269E298A297225811D
:0E9AF60025902572299E25AC25010000000058
:00000001FF
